:10A82F0047415445202D3E49533A20004741544556
:08A83F00202D3E52463A200094
:10A8E4007B017A007980227B017A00790090010053
:03A8F400E0FD2262
:10A00800300839C208C2B5E4FF1223B6EF64017004
:10A018002912A8E4125F91C2B612A8E412779F121F
:10A02800A8E41268DB7BFF7AA8792FE4FD1270C8D8
:0DA0380012A8E4E4FD1270C8D2B6D2B52221
:10A0B900300935C209C2B5E4FF1223B6EF64017055
:10A0C9002512A8EB1296F112A8EB127BBB12A8E499
:10A0D900125F917BFF7AA8793BE4FD1270C812A840
:09A0E900E4E4FD1270C8D2B522B6
:109CD4000D0A494F31202D3E544E433A2000575827
:109CE40020426F617264206E6F206C696E6B0D0A86
:109CF400000D0A494F32202D3E544E433A2000575E
:109D040058353120200041504554353100574944DD
:0B9D1400453120005749444532200033
:1088EC0074032FF582E43401F583E0FF900211E06C
:1088FC002400F582E43400F58322EFF0900211E0BD
:10890C0004F022EFF0900210E004F0A3E004F02257
:10891C00EFF0900214E004F022900210E02474F5C1
:10892C0082E43402F583E0FF22900210E024BAF5D1
:10893C0082E43402F583E0FF22900210E004F0227E
:10894C00900213E004F022900210E0248AF582E4F5
:10895C003402F583E0FF22900210E024B2F582E4A9
:10896C003402F583E0FF22900210E0FFC3227C006A
:10897C007D0A122EA2ED243022900215E025E02271
:10A5230030B322E4FFFE12A88EEF60197F927E0102
:10A5330012A88EEF700C12A00812A0B9129DFD0292
:06A543009E4212A3B022AB
:0523B60090020FEFF0A2
:1023BB00E4900211F0EF14602124FE6036240370C8
:1023CB004BE4900210F0900210E0909D0A93603C59
:1023DB0025E01288F712890F80ECE4900210F09040
:1023EB000210E0909D0393602325E01288F7128979
:1023FB000F80ECE4900210F0900210E0909D0A9395
:10240B00600A25E01288F712890F80EC1288F874A5
:10241B0060128907E4A3F0A3F0A3F01229FBEF608D
:10242B001A1229FBEF25E01288F712891C70031290
:10243B00894C128908A3E004F080E0900212E0C3FB
:10244B0094065025E4900210F0900212E0FFC37442
:10245B00069FFF900210E0C39F500EA31288FB74DF
:10246B004012890712894580E090020FE014601A30
:10247B0024FE60212403702E7F877E0012A88E908D
:10248B000215EFF07F847E0080147F07122A6A7F8B
:10249B00047E0180097F93122A6A7F947E0112A821
:1024AB008E900216EFF0900216E024FE602A047064
:1024BB007312898544E01288F7128906E4900210A2
:1024CB00F0900210E0909D1193600A25E01288F7BE
:1024DB0012890F80EC02252812898544E01288F7B7
:1024EB00128906E4900210F0900210E0909D119377
:1024FB00600A25E01288F712890F80EC1288F874B5
:10250B0062128907E4900210F0900210E0909D187F
:10251B0093600A25E01288F712890F80EC1288F875
:10252B007463800912898544611288F7EF12890759
:10253B001288F874031289071288FB74F01289074A
:10254B0090020FE0600302263D122A1F701E9002BC
:10255B0013F0A37490F0122A07EF60561229E212BF
:10256B00891C700312894C12890880EA1299C3EFF7
:10257B007002FF227F907E0012A88E1288F81289BB
:10258B0006E4900210F012892560081288F812896F
:10259B000F80F3900213E4F0A374A3F0122A07EF59
:1025AB0060101229E212891C700312894C128908DF
:1025BB0080EA7F857E0012A88EEF64017018128866
:1025CB00F87420128907122A75128935600812884F
:1025DB00F812890F80F3122A1F7022126A45EF64DA
:1025EB0001701A1288F87420128907E4900210F017
:1025FB0012895360081288F812890F80F3122A2867
:10260B00600302295112295F743A128907E4900280
:10261B0010F012896360081288F812890F80F31288
:10262B0088F874751289071288FB74671289070280
:10263B00295190020FE064016003022800122A580E
:10264B00707590021304F0A37410F0E4900210F074
:10265B00122A131288F812891C700312894C1289E2
:10266B0008128945E0C3941440E6E4FF1295A6EFE7
:10267B0070097BFF7A9C79D40227047A9C79D41257
:10268B002A331289739404500B1288EC12890612A8
:10269B00894580EE1288F8742F1289079002107406
:1026AB0005F0128973942140030227651288EC12FE
:1026BB00890612894580EB1299C3EF7002FF227FC6
:1026CB00107E0112A88E1288F8128906E49002106F
:1026DB00F012892560081288F812890F80F37F2386
:1026EB007E0112A88E1288F81289067F011295A618
:1026FB00EF702E7BFF7A9C79F5FD1270C87BFF7A09
:10270B009C79E2E4FD1270C87B017A007980E4FDCC
:10271B00123EF97B017A007980E4FD123B9E7F002B
:10272B00227A9C79F5122A331289739404500B1276
:10273B0088EC12890612894580EE1288F8742F12E4
:10274B0089079002107405F01289739421500B12B3
:10275B0088EC12890612894580EE9002137401F001
:10276B00A37445F0122A13EF6013122A4C1288F847
:10277B0012891C700312894C12890880E77F05129D
:10278B002A6170181288F87420128907122A7512A0
:10279B00893560081288F812890F80F3122A587055
:1027AB0022126A45EF6401701A1288F8742012899C
:1027BB0007E4900210F012895360081288F812890E
:1027CB000F80F3122A28702A12295F743A12890794
:1027DB00E4900210F012896360081288F812890FD6
:1027EB0080F31288F874751289071288FB746712CC
:1027FB00890702295190020FE0FEB402037F0122E8
:10280B00EE6403600302295C1288F87421128907B5
:10281B00E4900210F012892560081288F812890FD3
:10282B0080F37F977E0112A88E1288F81289067F9B
:10283B008E122A6160030228FD900252E0FAA3E097
:10284B00FB7C007D64FFAE02122EA2EF24301288B7
:10285B00F71289067C007D0AAF03AE02122EA2127C
:10286B00897AFF1288FB128906900252E0FEA3E0E0
:10287B00FF12897A1288F71289061288FB742F12BD
:10288B00890790025BE0FF75F064842430FE1288A8
:10289B00F8EE128907EF75F00A8475F00A84E5F0FB
:1028AB002430FF1288FB12890690025BE075F00A58
:1028BB0084E5F024301288F71289061288FB742FF6
:1028CB001289071288FB74411289071288FB743D29
:1028DB00128907E4900210F0128973940650137456
:1028EB00542FF582E434021288F4128906128945BA
:1028FB0080E69002137401F0A374B0F0122A4CEF2F
:10290B00601B900213E0FEA3E0FF12A88E1288F862
:10291B0012891C700312894C12890880DF7F987E04
:10292B000112A88EEF6401701D1288F874201289B1
:10293B0007128BF3E4900210F012893560081288AD
:10294B00F812890F80F3900211E0900100F07F01E3
:03295B00227F00D8
:10295E0022126E5B900211E02400F582E43400F541
:10296E00837420F0900211E004F0E02400F582E47C
:10297E003400F5837450F0900211E004F0E024006E
:10298E00F582E43400F583744DF0900211E004F00A
:10299E00E02400F582E43400F5837432F0900211E5
:1029AE00E004F0E02400F582E43400F583742EF0A8
:1029BE00900211E004F0E02400F582E43400F58387
:1029CE007435F0900211E004F0E02400F582E43456
:1029DE0000F58322900213E0FEA3E0FF12A88E9072
:1029EE000211E02400F582E43400F58322900213F4
:1029FE00E0FEA3E0FF12A88E22900213E0FEA3E0F9
:102A0E00FF12A88E22900213E0FEA3E0FF12A88E02
:102A1E00227F087E0112A88EEF227F347E0012A83C
:102A2E008EEF6401227BFFE4FD1270C87B017A01F8
:102A3E007903E4FD1270C89002107401F022900226
:102A4E0013E0FEA3E0FF12A88E227F087E0112A8DB
:102A5E008EEF227E0112A88EEF6401227E0112A853
:102A6E008E900215EFF022128BF3E4900210F022FA
:100026000D0A575820202D3E4953203A20000D0A2C
:0C003600575820202D3E5246203A200052
:10A73D007B017A007980227B017A0179037D0122E8
:0CA74D007B017A007900900100E0FD2201
:109DFD00300C41C20CC2B57F011223B6EF64017065
:109E0D003112A73D125F9112A73D12779F12A73D08
:109E1D001268DB7BFF7A007926E4FD1270C812A769
:109E2D003DE4FD1270C812A744123EF912A7441268
:059E3D003B9ED2B5229E
:10A4D500900103E064636007E4900185F0FF22903A
:10A4E5000185E064246004E4F0FF229002D2740147
:07A4F500F0E4F5AF7F012246
:109E4200300B41C20BC2B57F011223B6EF64017021
:109E52003112A74D1296F112A74D127BBB12A73DEC
:109E6200125F917BFF7A007934E4FD1270C812A769
:109E72003DE4FD1270C812A744123EF912A7441223
:059E82003B9ED2B52259
:1095A600E4F5AF90018404F0759CF4EF700543A2D6
:1095B600108003E4F5A2E49002D2F0900185F090C9
:1095C600022EF090022EE0FFC39480501774032FF2
:1095D600F582E43401F583E4F090022EE004F0E035
:1095E60004F080DF75AF01E490022EF09002D2E025
:1095F60070177F01FE12A70190022EE004F0E0D35F
:0E960600943240E8E4F5AFFF22E4F5AF7F01B7
:019614002233
:10A6A700202020202020202020202020200D0A00EC
:0EA6B7004750532D3E42454143454E3A200048
:10A54900900100E0FF90020EE0FEC39F2274002EEE
:10A55900F582E43400F583E0FF227B017A0079007B
:06A56900900100E0FD225C
:10808C00C2B51281687F031223B612A5631296F152
:10809C0012A563127BBB7FC012AA43E4FF12AA4352
:1080AC00E490020EF012A549500E12A55612AA43E6
:1080BC0090020EE004F080ED7FC012AA437B017A9F
:1080CC00007980125F917B017A00798012779F7B17
:1080DC00FF7AA679B71281521281521268DB7F8423
:1080EC007E0112A88EEF14600E14602614604624D4
:1080FC00037047E4FF8040E490020EF090020EE023
:10810C002480F582E43400F583E0FF602D12815E5B
:10811C0080EA7FC012A85FE4FF12A85FE490020E11
:10812C00F012A549500812A55612815E80F37FC04B
:10813C0012A85F80057F01124BB8128168125DCBCB
:05814C00124DE9D2B55F
:1081510022E4FD1270C87B017A0079802212A85FA7
:1081610090020EE004F0227BFF7AA679A7E4FD12CB
:0381710070C822B1
:108847000D0A50494E47204641494C2C5345525634
:108857004552204F46464C494E45200D0A000D0A09
:10886700534552564552204C494E4B205354415282
:10887700542E2E2E0D0A0053455256455220434C76
:108887004F534520210D0A00534552564552205457
:1088970043502F4950204C494E4B204F5554544973
:1088A7004D45210D0A005345525645522054435019
:1088B7002F4950204C494E4B204F555454494D4554
:1088C700203E2033202C4E6F7720544E4320526594
:1088D70073657420210D0A0075736572200020707E
:0588E700617373200025
:1090F10090022AE02480F582E43400F58322900274
:109101001BE0FEA3E0FF900219E0FCA3E0FD90024A
:1091110016E02DFD900215E03CFC22F090022AE0C1
:1091210004F022EFF0900229E004F0A3E004F02221
:1091310090020F7404F0A3E4F0223400FEF0A3EFD8
:10914100F0EE5407FEE42FFFEE344022FF90021BA5
:10915100E03400FE22EFF0900226E004F022340019
:10916100F0A3CEF022900225E004F022900225E443
:03917100F0A32246
:1064560090021B1291342402FFE43404FE12A2FDC2
:10646600900211EFF07D0212000EEF64016003024C
:1064760065CB90021CE0240212914D900211E0447B
:1064860004FD12A59B90021CE024261265CC7F0019
:10649600FEC006C00790021CE024271265CCFDD082
:1064A600E02DFED0E090021912915F90021CE024CC
:1064B6002812914D12A2FDEF7F00FEC006C0079084
:1064C600021CE0242912914D12A2FDEFFDD0E02D11
:1064D600FED0E090021512915FD390021AE09480EC
:1064E600900219E0940040061290FF029F4E90021F
:1064F60015E05407FEA3E02400FFEE3460A3F0A3EA
:10650600EFF0A3E0FFA3E0900213CFF0A3EFF0E4D7
:10651600900212F0900213E07002A3E0604C900229
:1065260017E0FEA3E0FF12A2FD9002121290F4EF14
:10653600F0900218E004F07006900217E004F09064
:106546000212E004F0900214E024FFF0900213E03F
:1065560034FFF0900217E0B468BAA3E0B400B59037
:1065660002177460F0A3E4F080AA9002121290F46D
:10657600E4F01290FF129F4E7B017A007980E4FDD1
:106586001270C8900080E0642370339002C4F0203B
:106596001233900212F0FF9002121290F4E0FE60A5
:1065A6000EB420010F900212E004F0EFB403E8905D
:1065B60002121290F4E0B47602D21202473FC2B53C
:0565C600126F95D2B533
:0E65CB0022FF90021BE03400FE12A2FDEF2220
:10A941009002C4E004F0E0D3943C4004E4F0D2135C
:01A9510022E3
:10A6C5009002C3E0FFB4020F0512E512D3940240D5
:0EA6D5000CE4F512B2B722EFB40302B2B722C2
:10A6E3001271F39002C57413F0A37488F07513010B
:0EA6F300E49002C2F0A3F0F512A3F0C213220D
:10A9520020C303025647E49002C3F0D2B7D2B62214
:10A29D009002C6E004F070069002C5E004F0D39081
:10A2AD0002C6E0948D9002C5E0941340137413F030
:10A2BD00A37488F00513E513D394034003751301BC
:01A2CD00226E
:105647001291313013159002C4F0C21312A29DE4D7
:105657009002C3F07A88794712583F9002C3E060FE
:10566700030257617A88796512583F129131D2B790
:10567700C211C2129002C4F0C213FF12581790024F
:10568700C5E0FD7404FFFE12A59B9002C5A3E0FDD3
:105697007F057E0412A59B7F0112581712580A64D2
:1056A7001360030257587F2FFE12A88EEF64017014
:1056B700057F22FE800DE51324FE602304703C7FE6
:1056C700227E0012A88EAD0712581F7F231257D6CD
:1056D7001258277F241257D612582F7F2580427FD2
:1056E700261257FA12581F7F271257FA1258277F88
:1056F7002812580212582F7F2980267F2A12580213
:105707007F0C7E0412A59B7F2B1258377F0D7E04DA
:1057170012A59B7F2C1258377F0E7E0412A59B7F04
:105727002D7E0012A88EAD077F0F7E0412A59B7DEC
:10573700387F107E0412A59B7DF47F117E0412A58D
:105747009B7D047F017E0412A59B9002C37401F028
:10575700227D107F017E0402A59B12580ABF1713F2
:105767009002C32012057403F080057405F0C2B7D8
:105777000264569002C37402F0FF7E0412A2FD90E9
:10578700020EEFF030E10EE044021257DE7A88791C
:105797007EFD0270C890020EE030E33244081257D3
:1057A700DE7A88798FFD1270C87F307E0012A88E4E
:1057B700BF011B9002C2E004F0E0D39403400FE462
:0E57C700F07BFF7A8879ADFD1270C875C7209F
:1057D500227E0012A88EAD0722FD7F027E0412A54F
:1057E5009B7D107F017E0412A59B12A29DE4900271
:1057F500C3F07BFF227E0012A88EAD07227E001229
:10580500A88EAD07227F037E0412A2FD90020DEF44
:10581500F0227D017E0412A59B227F0C7E0412A539
:105825009B227F0D7E0412A59B227F0E7E0412A56E
:105835009B227E0012A88EAD07227BFFFD1270C849
:015845002240
:10473F0030110302494DE4FFFE12A88EEF70030201
:10474F00494D7F0912497F700302494DE490022AB7
:10475F00F0900229F0900229E09088DF93FF600823
:10476F001290F112912480EDE4900225F0A3F01243
:10477F00494EEF601312494E1290F1129156700389
:10478F0012916612911D80E77F0712497F603012E8
:10479F0090F1742D12911CEFC3940AEF5002801503
:1047AF0075F00A842430FE1290F1EE12911CEF7511
:1047BF00F00A84E5F02430FF1290F4EF12911CE41C
:1047CF00900229F0900229E09088E593FF6008128B
:1047DF0090F112912480ED12916D7409F012495AE3
:1047EF00EF601312495A1290F11291567003129101
:1047FF006612911D80E7E4900229F0900229E09063
:10480F00A56F93FF60081290F112912480ED129121
:10481F006D7440F0FF7E0012A88EEFC394FF501FFF
:10482F0012916D7440F0124973EF601312497312B5
:10483F0090F1129156700312916612911D80E7123A
:10484F0090F1740D12911C1290F4740A12911C12B3
:10485F0090F4E4F09002271291342420FFE4340402
:10486F00FE12A2FDEF7F00FEC006C007900228E0F7
:10487F002421124966FDD0E02DFED0E034009002D5
:10488F001FF0A3CEF0900228E024241249667F0087
:10489F00FEC006C007900228E02425FF900227E003
:1048AF003400FE12A2FDEFFDD0E02DFFD0E090020C
:1048BF001D12913B900221F0A3EFF0E4A3F0A3F0BF
:1048CF00900229F09002291290F4E0FD60449002CA
:1048DF0021E0FEA3E0FF12A59B900222E004F070FE
:1048EF0006900221E004F0900229E004F0900224E7
:1048FF00E004F07006900223E004F0900221E0B48F
:10490F0048C2A3E0B400BD9002217440F0A3E4F0CC
:10491F0080B2900227E0FEA3E0FF900223E0FCA309
:10492F00E0FD90021EE02DFD90021DE03CFC12A266
:0E493F00057B017A007980E4FD1270C8D21168
:10494D0022900225E0FEA3E0FF12A88E2290022500
:10495D00E0FEA3E0FF12A88E22FF900227E03400B4
:10496D00FE12A2FDEF22900225E0FEA3E0FF12A8A9
:09497D008E227E0012A88EEF22AA
:0B779F0090020FEBF0A3EAF0A3E9F06A
:1077AA009002C3E06405600302789FC2B690021A91
:1077BA001291342420FFE43404FE12A2FDEF7F006C
:1077CA00FEC006C00790021BE024211278A0FDD05B
:1077DA00E02DFED0E03400900216F0A3CEF0900225
:1077EA001BE024241278A07F00FEC006C007900286
:1077FA001BE02425FF90021AE03400FE12A2FDEFDE
:10780A00FDD0E02DFFD0E090021412913B900218B7
:10781A00F0A3EFF0E4900212F0A3F090020FE0FB65
:10782A00A3E0FAA3E0F9122E28FD6048900218E0BE
:10783A00FEA3E0FF12A59B900219E004F0700690E7
:10784A000218E004F0900210E475F001122EF7908D
:10785A000213E004F07006900212E004F09002189D
:10786A00E0B448B7A3E0B400B29002187440F0A3A1
:10787A00E4F080A790021AE0FEA3E0FF900212E073
:10788A00FCA3E0FD900215E02DFD900214E03CFC03
:05789A0012A205D2B6A8
:0E789F0022FF90021AE03400FE12A2FDEF223A
:109454002348454C4C4F002352455345540023495F
:109464004E5354414C4C0023474154455F52465F90
:10947400544553540023474154455F49535F544571
:109484005354002357585F52465F544553540023A6
:1094940057585F49535F54455354000D0A00632ED7
:1094A4002E2E732E2E2E672E2E2E742E2E2E722ED0
:1094B4002E2E702E2E2E682E2E622E2E2E2E2E0D39
:0294C4000A009C
:108FE900900212E05407FEA3E02400FFEE347090D3
:108FF90002CCF0A3EFF07BFF2290021EE0FBA3E07E
:10900900FAA3E0F9022E2890022CE475F001022E51
:10901900F73400FEF0A3EFF0EE5407FEE42FFFEE65
:10902900345022FF90021CE03400FE229002CCF062
:10903900A3E4F022EBF0A3EAF0A3E9F0227406F02E
:10904900A3E4F02420FFE43406FE22E49002CBF0EE
:10905900C219223400F0A3CEF0229002347450F0E9
:04906900A3E4F0226A
:0AAA390020C303028DAF12905422D7
:03AA8600C21922D0
:1050170090021C7406F0A3E4F02402FFE43406FEB9
:1050270012A2FD900210EFF07D0212000EEF640154
:1050370060030251D890021DE0240212902C9002C6
:1050470010E04404FD12A59B90021DE02426125295
:10505700157F00FEC006C00790021DE024271252EC
:1050670015FDD0E02DFED0E090021412905C900266
:105077001DE0242812902C12A2FDEF7F00FEC0062F
:10508700C00790021DE0242912902C12A2FDEFFD0B
:10509700D0E02DFFD0E03400900212F0FCA3EFF037
:1050A700FD900215E02DFE900214E03C900216F0F0
:1050B700A3CEF0EC5407FEE42F128FF47A947954C0
:1050C70012A622EF6401707C900214E07004A3E042
:1050D7006406700BC2AC1251D9124986D2AC229029
:1050E7000214E064027004A3E064067057C2AFC202
:1050F700B4C2B5FFFE12A90AE490021AF0A3F09019
:105107000218F0A3F012A385900211EFF0FD9002B0
:105117001AE0FEA3E0FF12A5E390021BE004F07083
:105127000690021AE004F0900219E004F07006906D
:105137000218E004F0C3900218E0940240C712512D
:10514700D975C720128FE97A94795B12A622BF011D
:10515700061251ED75C720128FE97A94796212A66B
:1051670022BF01091251ED125A2375C720128FE988
:105177007A94796B12A622BF0106125201D2092234
:10518700128FE97A94797912A622BF010612520189
:10519700D20822128FE97A94798712A622BF010BCF
:1051A70090021CE0FE125222D20B22128FE97A944F
:1051B700799312A62290021CE0FEBF01061252222A
:1051C700D20C22A3E0FF900216E0FCA3E0FD129FA1
:0151D7004E89
:1051D8002290021CE0FEA3E0FF900216E0FCA3E090
:1051E800FD129F4E2290021CE0FEA3E0FF900216E3
:1051F800E0FCA3E0FD129F4E2290021CE0FEA3E01B
:10520800FF900216E0FCA3E0FD129F4E22FF9002E1
:105218001CE03400FE12A2FDEF22A3E0FF9002166C
:09522800E0FCA3E0FD129F4E2200
:10A385009002CCE0FEA3E0FF12A2FD9002CDE00416
:10A39500F070069002CCE004F09002CCE0B4780AAC
:0AA3A500A3E0B400057470129035B7
:01A3AF00228B
:10A32B00AD079002CCE0FEA3E0FF12A59B9002CDFF
:10A33B00E004F070069002CCE004F09002CCE0B4A4
:0DA34B00580AA3E0B40005745012903522AA
:10A6220090021E12903D129002601412A3851290A5
:10A63200026F60037F002290021F12901380E77F57
:02A642000122F3
:06A45A0090022E12903D5D
:10A46000E4A3F090022E129005FF601112A32B902E
:10A47000022F129013900231E004F080E690023136
:02A48000E0FFFB
:01A4820022B7
:10498600C2B690022C12904612A2FDEF7F00FEC026
:1049960006C00790022DE02421124B80FDD0E02DA9
:1049A600FED0E090022A12905C90022DE0242412A0
:1049B6004B807F00FEC006C00790022DE02425FF35
:1049C60090022CE03400FE12A2FDEFFDD0E02DFF98
:1049D600D0E090022812901A9002CCF0A3EFF0E4F7
:1049E600900222F0A3F07BFF7A947954124B8DE467
:1049F600900224F0A3F0900220F0A3F0900224E0AD
:104A0600FEA3E0FF12A88E90021EEFF012A32B90D9
:104A16000225E004F07006900224E004F0900221E2
:104A2600E004F07006900220E004F0C3900220E05B
:104A3600940240C8900223E02400F0900222E03461
:104A460002F07AA5796F124BA3EFF07A94799F1250
:104A56004BA3E004F0E004F0E513124B0DE49002E2
:104A66001FF09002C5E0FEA3E0FF900226EEF0A341
:104A7600EFF07C037DE8122EA2EF124BACF07D64C2
:104A8600124B3B7D0A124B3B900226E0FEA3E0FF51
:104A96007C007D0A122EA2ED124B0DE490021FF04F
:104AA6009002C3E0124BAC124B5D129ECCEF640138
:104AB6007017FF1295A6BF01087B017A0179038062
:104AC6000E7BFF7A9479A280067BFF7A9479A212F4
:104AD6004B8D128BF37B017A0279BA12A45A90029B
:104AE6001FEF124B5D90022CE0FEA3E0FF90022226
:104AF600E0FCA3E0FD900229E02DFD900228E03CB9
:064B0600FC12A205D2B66C
:104B0C00222430FF12A32B90021FE004F07BFF7ACB
:104B1C0094799F12A45A90021FE004F0E004F0E094
:104B2C00FF900223E02FF0900222E03400F022905C
:104B3C000226E0FEA3E0FF7C00122EA27C007D0A80
:104B4C00122EA2ED2430FF12A32B90021FE004F0D2
:104B5C0022F07BFF7A94799F12A45A90021FE004F2
:104B6C00F0E004F0E0FF900223E02FF0900222E04E
:104B7C003400F022FF90022CE03400FE12A2FDEF74
:104B8C002212A45A90021FEFF0900223E02FF09013
:104B9C000222E03400F0227BFF12A45A90021F2262
:0C4BAC002430FF12A32B90021FE0042213
:109ECC007F00129F0340037F01227401FFFE12A842
:109EDC008EEFD3940040037F01227F02129F034038
:109EEC00037F01227F037E0112A88EEFD3940040E2
:109EFC00037F01227F00227E0112A88EEFD39400F3
:019F0C002232
:108DAF0090020E7406F0A3E4F020193C129055D2F5
:108DBF00B67D01FF7E0612A59B7DEA7F047E06121B
:108DCF00A59B7D607F057E0612A59B7D01128E2BD4
:108DDF00BF130C7D02128E2B6414703FD219227DAB
:108DEF00107F017E0602A59B7F037E0612A2FD90D7
:108DFF00020DEFF0601724E4600F2405701D900240
:108E0F00CB7401F0C2B60250177D0880027D107F2F
:0B8E1F00017E0612A59B129054D2B6F3
:108E2A00227F017E0612A59B7F037E0612A2FD9079
:058E3A00020DEFF02223
:0970C80090022B12903DA3EDF0A3
:1070D1009002CBE070030271DB90023612904612EF
:1070E100A2FDEF7F00FEC006C007900237E0242119
:1070F1001271DCFDD0E02DFED0E03400900232F0C0
:10710100A3CEF0900237E024241271DC7F00FEC090
:1071110006C007900237E02425FF900236E03400D4
:10712100FE12A2FDEFFDD0E02DFFD0E09002301263
:10713100901A900234F0A3EFF090022EE07038A381
:10714100F090022B129005FD6073900234E0FEA3D3
:10715100E0FF1271E97006900234E004F012901021
:1071610090022FE004F0900234E0B458D4A3E0B4CC
:1071710000CF12906380CA90022EE0A3F090022FFC
:10718100E06034900234E0FEA3E0FF90022B129005
:1071910005FD1271E97006900234E004F0129010BE
:1071A10090022FE014F0900234E0B458D0A3E0B480
:1071B10000CB12906380C690022EE0A3F0900236BD
:1071C100E0FEA3E0FF90022FE0FD900231E02DFDF3
:0A71D100900230E03400FC12A20529
:1071DB0022FF900236E03400FE12A2FDEF2212A530
:0871EB009B900235E004F02244
:10A8D000FF900214E03400FE227407F0A3E4F0902D
:04A8E00002D5E0229B
:0CA9FD0020C303029270E49002D5F02207
:06AA7B00E49002D5F02278
:1083F9009002147407F0A3E4F02402FFE43407FEAA
:1084090012A2FD900211EFF07D0212000EEF64013D
:1084190060030284B0900215E0240212A8D09002F1
:1084290011E04404FD12A59B900215E02426128454
:10843900B17F00FEC006C007900215E02427128410
:10844900B1FDD0E02DFED0E03400900212F0A3CEB1
:10845900F0900215E0242812A8D012A2FDEF7F00A7
:10846900FEC006C007900215E0242912A8D012A266
:10847900FDEFFDD0E02DFFD0E03400AD07FC54073F
:10848900FEE42FFFEE3478FEE4B50704EEB4800075
:10849900900214E0FEA3E0FF900213E02DFD90028C
:0784A90012E03CFC129F4EA3
:0E84B00022FF900214E03400FE12A2FDEF2223
:109270007F317E0012A88EEF606F90020F12A8D986
:10928000703F7D02FF7E0712A59B7DEA7F047E076B
:1092900012A59B7D6A7F057E0712A59B7D017F013C
:1092A0007E0712A59B7F037E0712A2FDBF220990B5
:1092B00002D57401F00283F97D107F017E0702A5BB
:1092C0009B7F027E0712A2FDEF30E31D90020DA3EB
:1092D000E04408FD7F027E0712A59B7D107F017E82
:0992E0000712A59BE49002D5F0F1
:0192E9002262
:0B68DB0090020FEBF0A3EAF0A3E9F03D
:1068E6007F317E0012A88EEF7003026A2A90021A88
:1068F60012A8D97003026A2A7F037E0712A2FDEF4F
:1069060064226003026A2AC2B67DDA7F0C7E071211
:10691600A59B7D687F0D7E0712A59B7DB17F0E7EB0
:106926000712A59B7DD37F0F7E0712A59B7D387F1F
:10693600107E0712A59B7DF47F117E0712A59B9002
:10694600021BE02420126A2B7F00FEC006C00790BF
:10695600021BE02421126A2BFDD0E02DFED0E0348C
:1069660000900216F0A3CEF090021BE02424126AD7
:10697600387F00FEC006C00790021BE02425126A7D
:1069860038FDD0E02DFFD0E03400FE900214F0A3D5
:10699600EFF0EE5407FEE42FFFEE3458900218F0A5
:1069A600A3EFF0E4900212F0A3F090020FE0FBA335
:1069B600E0FAA3E0F9122E28FD6048900218E0FEE6
:1069C600A3E0FF12A59B900219E004F07006900266
:1069D60018E004F0900210E475F001122EF7900210
:1069E60013E004F07006900212E004F0900218E042
:1069F600B460B7A3E0B400B29002187458F0A3E4F0
:106A0600F080A790021AE0FEA3E0FF900212E0FCDD
:106A1600A3E0FD900215E02DFD900214E03CFC126F
:046A2600A205D2B63D
:106A2A0022FF90021AE03400FE12A2FDEF22FF902C
:0B6A3A00021AE03400FE12A2FDEF2261
:09AA5700FF900238E03400FE22F9
:10000E00AE05EFA806088002C313D8FC30E0037FCC
:05001E0001227F002219
:1071F300D294C297C28312A99ED2837F101272DEE9
:107203007F0F7E0012A59B7F111272DE7F107E001E
:1072130012A59B7F121272E67F117E0012A59B7F3F
:10722300131272E67F127E0012A59B7F141272EE78
:107233007F057E0012A59B7F151272EE7F067E00EE
:1072430012A59B7F161272F67F077E0012A59B7F05
:10725300171272F67F087E0012A59B7F181272FE2A
:107263007F017E0012A59B7F191272FE7F027E00B2
:1072730012A59B7F1A1273067F037E0012A59B7FC4
:107283001B1273067F047E0012A59B7F1C12730ED4
:107293007F097E0012A59B7F1D12730E7F0A7E005D
:1072A30012A59B7F1E1273167F0B7E0012A59B7F78
:1072B3001F1273167F0C7E0012A59B7F207E001287
:1072C300A88EAD077F0D7E0012A59B7F217E001245
:1072D300A88EAD077F0E7E0002A59B7E0012A88EAE
:1072E300AD07227E0012A88EAD07227E0012A88E63
:1072F300AD07227E0012A88EAD07227E0012A88E53
:10730300AD07227E0012A88EAD07227E0012A88E42
:0B731300AD07227E0012A88EAD0722FD
:0EA99E00E4F5D875F9FDF5E9D2DE30DFFD22D3
:10A7C700E4FEEF30E704D2958002C295D297EF25D9
:09A7D700E0FFC2970EEEB408E9A0
:01A7E0002256
:07A59400FFE43EFEA3E0FD21
:10A59B00AB07AA06C2947FF012A7C7EAFF12A7C7A0
:0DA5AB00AF0312A7C7AF0512A7C7D29422B5
:04A2FD00AD07AC06F7
:10A30100C2947F0F12A7C7ECFF12A7C7AF0512A710
:10A31100C7E4FFFED297EF25E0FF3096034401FF2B
:09A32100C2970EEEB408EDD294CF
:01A32A002210
:10A2050090023AECF0A3EDF0900238EEF0A3EFF0F7
:10A21500242412A594900239E0242512AA5790020D
:10A225003BE0FD12A59B900239E0240112AA577D5F
:04A235002002A59BC3
:109F4E00900220ECF0A3EDF090021EEEF0A3EFF0E5
:109F5E00242812A59490021FE02429FF90021EE0EF
:109F6E003400FE900221E0FD12A59B90021FE0241A
:0E9F7E0001FF90021EE03400FE7D4002A59B14
:109C8700E0FAA3E0FBFFAE02122EA2EF2430FF9012
:109C97000217E0248AF582E43402F583EFF090029C
:109CA70017E004F0227C00AF03AE02122EA27C0064
:109CB7007D0A122EA2ED22E0248AF582E43402F511
:0D9CC7008322E0FAA3E0FB7C007D0AFF226F
:106A450012A406EF7002FF227FCC12A7597F4412D1
:106A5500A7593092FD12A406EF7002FF227FCC12D7
:106A6500A7597FBE12A75912A644900292E4F0A33B
:106A7500EFF012A644900290E4F0A3EFF0E4900248
:106A850017F0900217E0FFC39406500C748A2F127A
:106A95009CC1E4129CA480EA900290A3E0FF30E739
:106AA5001DD21AFE900293E02400FF900292E03E70
:106AB500FEEFF4FFEEF4FEEF2401FDE48012C21AAE
:106AC500900291E0FE900293E02400FD900292E096
:106AD5003EFCE4122C29E4FBFA7920783F122A7E49
:106AE500122C62900218EEF0A3EFF0E4900217F07A
:106AF500301A08129CBE742D129CA4C3900219E092
:106B05009464900218E09400500C129CC9AE0212D5
:106B15002EA2EF026B7EC3900219E094E890021852
:106B2500E09403502C7C007D64129C877D0A129CA6
:106B3500AC2430FF129C99129CBE742E129CA4A307
:106B4500E0FEA3E0FF129CB52430FF900217026B14
:106B550098C3900219E09410900218E094275041D0
:106B65007C037DE8129C877D64129CAC2430FF1267
:106B75009C99A3129CC9129CB0129C93129CBE7442
:106B85002E129CA47C007D0AAF03AE02122EA2ED4C
:106B95002430FF129C99129CBE7443129CA47F0161
:036BA500227F004C
:016BA80022CA
:07A91D0012A924D2927F0170
:0BA92400AE071FEE6004000080F6226A
:10A40600D2D7C2927FF012A9247FF012A924D29249
:10A416007F3C12A924A2927FF012A9247FB412A92C
:0AA426002420D7037F01227F0022CB
:10A64400E4FDFCEDC313FDC2927F0112A91D3092FB
:10A6540004ED4480FD7F3C12A9240CECB408E4AF63
:01A6640005F0
:01A6650022D2
:02A75900AD074A
:10A75B00E4FCC2927F0112A924EDC313FD92927FF8
:09A76B003C12A91D0CECB408E934
:01A7740022C2
:10A239007C00AF03AE02122EA27C007D0A122EA270
:10A24900ED2430FFE024B2F582E43402F583EFF027
:10A25900900217E004F022E024B2F582E43402F51A
:02A2690083224E
:106E5B00E4900217F0C282E4F5D875F9FE75E9FEED
:106E6B00D2DE30DFFDE4FF12A12A900218EEF0A370
:106E7B00EFF0E4F5D875F9FF75E9DBD2DE30DFFD15
:106E8B00D282E4F5D875F9DD75E927D2DE30DFFD66
:106E9B0012A259E0C3943240BC900218E0FCA3E06C
:106EAB00FDE4122C297B337A3379537840122A7EF6
:106EBB00E4FBFA79807844122B87E4FBFA79A0780B
:106ECB0041122A7E122C62E4900217F0900217E016
:106EDB00FDC39408500C74B22D12A263E412A25895
:106EEB0080EAD3EF9406EE94005003026F77EF2401
:106EFB00FAFFEE34FFFEEFC4F8540FC868FFEEC480
:106F0B0054F048AB07FAE4900217F07C037DE8AE2F
:106F1B0002122EA2EF12A24A7D6412A2397D0A122E
:106F2B00A2397C007D0AAF03AE0212A246C3EB94DA
:106F3B0064EA940050119002B4E09002B2F0900217
:106F4B00B5E09002B38020C3EB94E8EA9403503988
:106F5B009002B3E09002B2F09002B4E09002B3F072
:106F6B009002B5E09002B4F0E4A3F022E490021793
:106F7B00F012A260742D12A25812A260742D12A2EC
:096F8B005812A260742D12A258E4
:016F940022DA
:0CAA090049532020202D3E52463A2000E8
:109F8C00F00C74002CF582E43400F58374A0F00C12
:109F9C0074002CF582E43400F5832274802DF58254
:109FAC00E43400F583E02274812EF582E43400F56C
:0E9FBC0083E022EEF00C90021DE004F00D2276
:109B3900E4FF74802F129FAA643E600A0FEFD3944A
:109B49000C40EF7F6322E4FE74802E129FAAFD640D
:109B59003E6030ED642D7028C3EF9EB40208129F59
:109B6900B3C39430FF22129FB324D075F00AA4FF27
:109B790074822EF582E43400F583E024D02FFF228D
:059B89000E80C57F0005
:019B8E0022B4
:0DA9D6007F2E7E0012A88E9002D6EFF02298
:106F95009002D6E070030270C7129B39EF646370EC
:106FA500030270C7E4FE74802E129FAA643E600837
:106FB5000EEED3940C40EF227D069000007440F055
:106FC500A3DDFC7D060EE4FC74802E129FAAFB64F3
:106FD5002C6012EB25E0FB129F9CEBF00C0EEED320
:106FE500941240E4229000067460F00C7D06900037
:106FF500077440F0A3DDFC7C07EFD39400401AE44E
:10700500FD90021DF0129FA7FE642D6026EE25E07F
:10701500FE129F9C129FBF80ECE4FD90021DF012B2
:107025009FA7FE643E600CEE25E0FE129F9C129F1A
:10703500BF80ECEF25E0446090000DF07C0E129FC0
:107045009C74A8129F9A7486129F8C7492129F8CBE
:107055007440129F9A74E1129F9A7403129F9A7456
:10706500F0F00CE4FD129FA7643A60080DEDD3948F
:107075003240F2220D129FA7FF6009129F9CEFF08C
:107085000C0D80F1AF04900100EFF0FD7B017A005B
:1070950079001296F17B017A007900900100E0FDFC
:1070A500127BBB7B017A007980125F917BFF7AAA04
:1070B5007909E4FD1270C87B017A007980E4FD123C
:0270C50070C891
:0170C70022A6
:1094C600E0FF90021EE0FBA3E0FAA3E0F99002227F
:1094D600E0F58275830022EF122E6E900222E004E0
:1094E600F02274002FF582E43400F583E0C3139074
:1094F6000224F0642022EF4430FFF090021EE0FBCD
:10950600A3E0FAA3E0F922E0541EC313900225F06B
:10951600D3940022900225E024F6F0E04430222481
:1095260006F582E43400F58322900221E004F0225D
:0B5F910090021EEBF0A3EAF0A3E9F081
:105F9C00E4900222F09002217407F0900221E0FFBD
:105FAC00C3940D50101294E860061294C61294DD3E
:105FBC0012952F80E690000D12950D402A1294C870
:105FCC00742D1294DE900225E0FFC3940A50051242
:105FDC0094FC800D1294C874311294DE12951AFF41
:105FEC00F01294D31294DD1294C8743E1294DEE431
:105FFC00900221F0900221E0FFC3940650101294FD
:10600C00E860061294C61294DD12952F80E690007B
:10601C000612950D402A1294C8742D1294DE90022B
:10602C0025E0FFC3940A50051294FC800D1294C80D
:10603C0074311294DE12951AFFF01294D31294DD7F
:10604C009002237407F090000DE030E0030260F73B
:10605C001294C8742C1294DEA3E02407F0E0900292
:10606C0021F0900223E02406FFE433FE900221E0AD
:10607C00FDC39FEE6480F8748098501374002D1249
:10608C0094EB60061294C61294DD12952F80D39077
:10609C000223E0FF12952512950D402F1294C8741F
:1060AC002D1294DE900225E0FEC3940A5009EE44B2
:1060BC0030FE129500800D1294C874311294DE12C9
:1060CC00951AFEF01294D3EE1294DE74062F1295EC
:1060DC0027E030E7081294C8742A1294DE90022349
:1060EC00E0129525E020E00302605C1294C8743A3B
:1060FC001294DEA3E02409F0E0900221F09001005C
:10610C00E0FF900221E0FEC39F501574002EF58233
:10611C00E43400F5831294C61294DD12952F80DDC1
:10612C001294C8740D1294DE1294D6740A1294DE72
:07613C001294D6E4022E6E5E
:10A8A50054544C2D3E4741524D494E3A20002447C1
:06A8B5005057504C2C002E
:10A0F200F583E0FF900211E02480F582E43400F55C
:10A102008322742CF0900211E004F022900210E0FD
:10A1120004F022900211E0FF900210E0FEC322F54B
:08A1220082E43400F583E02221
:054BB80090020FEFF078
:104BBD00900212740DF0E4A3F0900213E0C394037D
:104BCD004003024DE8900212E0240012A12120E0E2
:104BDD0003024DDBE4900211F0900210F0900210F0
:104BED00E0FFC394075011EF90A8B39312A0F5EF17
:104BFD0012A10612A10E80E5900212E0240490028B
:104C0D0010F0900212E0240BFFE433FE900210E04E
:104C1D00FDC39FEE6480F8748098501474002DF5D8
:104C2D0082E4340012A0F2EF12A10612A10E80D27E
:104C3D0012A0F612A104A3E0FF240BF582E43400C8
:104C4D00F583E0FE12A0F6EE12A10612A0F912A154
:104C5D0004EF240D900210F0900212E0FF2415FDD8
:104C6D00E433FC12A11A9DEC6480F8748098501303
:104C7D0074002E12A121FE12A0F6EE12A10612A1B1
:104C8D000E80D512A0F612A10474152FF582E4340E
:104C9D000012A0F2EF12A10612A0F912A1049002C7
:104CAD00107407F0900210E0FFC3940D50197400BA
:104CBD002F12A121C313FF6420600712A0F6EF127B
:104CCD00A10612A10E80DD90000DE0541EC313FF4E
:104CDD00D39400403012A0F6742D12A106EFC394A8
:104CED000AEF5002801575F00A842430FE12A0F6EA
:104CFD00EE12A106EF75F00A84E5F02430FF12A044
:104D0D00F9EF12A10612A0F6742A12A106E4FF9083
:104D1D00021004F0900211E0FE14FD900210E0FC70
:104D2D00C39D500E74802C12A0FCE06FFF12A10EDB
:104D3D0080E2EFC4540FFDC3940AED500C2430FDF6
:104D4D0074802E12A0FCED80072437FE12A0F6EE23
:104D5D0012A106EF540FFFC3940AEF5004243080C4
:104D6D0002243712A0F5EF12A10612A0F6740D124F
:104D7D00A10612A0F9740A12A10612A0F9E4F0908E
:104D8D00020FE07018A3F012A1159F502B74802E06
:104D9D0012A0FCE0FF12A84712A10E80EAE49002D7
:104DAD0010F012A1159F501074802E12A0FCE0FF80
:104DBD0012A85F12A10E80EA7BFF7AA879A5E4FD07
:104DCD001270C87B017A007980E4FD0270C89002F0
:0B4DDD0012E02407F012A10E024BC6EA
:014DE80022A8
:0EA9AC000D0A5246202D3E544E43203A200004
:10A7E100900100E0FF90020EE0FEC39F2274002E54
:0AA7F100F582E43400F583E0FF2256
:10832E00C2B4C2847FC012AA43E4FF12AA43E490EF
:10833E00020EF012A7E1500E12A7EE12AA439002FF
:10834E000EE004F080ED7FC012AA437B017A007923
:10835E0080125F917B017A00798012779F7BFF7A82
:10836E00A979AC1283E31283E31268DB7F847E016A
:10837E0012A88EEF14600E1460261460462403704B
:10838E0047E4FF8040E490020EF090020EE024805D
:10839E00F582E43400F583E0FF602D1283EF80EA6E
:1083AE007FC012A85FE4FF12A85FE490020EF012E5
:1083BE00A7E1500812A7EE1283EF80F37FC012A838
:1083CE005F80057F01124BB81244F2125231D2B4C3
:0583DE00D28402A8F7A3
:1083E300E4FD1270C87B017A0079802212A85F90A5
:0683F300020EE004F0227E
:109A2300F8900231E0FCA3E0FDA3E0FEA3E0FF1207
:109A33002F98E47B0AFAF9F8122F98EB2430FF9061
:109A43000239E024BAF582E43402F583EFF09002A0
:109A530039E004F0E024BAF582E43402F583227B92
:109A6300E87A03F9F8900231E0FCA3E0FDA3E0FEFD
:0E9A7300A3E0FF022F98F0900239E004F022E9
:0DA9E300759103759203759D0375BCA0224C
:10A12A00E4F5BDF5BEE5BC54E044084FF5BC0000BB
:10A13A0000007DFAE5BC30E41753BCEFAFBDEF7504
:10A14A00F004A4FFACBEEC7A002FFFEA35F0FE2241
:06A15A00DDE27E037FFF41
:01A1600022DC
:108BF3007F0112A12AE4FCFD900235123075E47F57
:108C0300E87E80FDFC900235E0F8A3E0F9A3E0FAEA
:108C1300A3E0FB122F0DE4FB7A24F9F8122F98EF4F
:108C23002423FFE43EFEE43DFDE43CFC90023112CC
:108C33003075E4129A62E4FBFAF9F8C31230387023
:108C430008900239F07B64801BE4900239F0129A99
:108C530062EF2430FF900239129A57EF129A79E4A7
:108C63007B64FAF9129A23742E129A79E47B0AFA36
:108C7300F9129A237456129A79900239129A57E488
:038C8300129A79C9
:018C860022CB
:10A7FB00E4F5D875F9FDF5E9D2DE229002CFE0C37E
:0AA80B0013F0229002CEE064032255
:10A7910020B317C2AC1287A190020DEFF012A815D9
:0AA7A10090020DE0B4010312832EB4
:01A7AB00228B
:1087A100128A2B12A80E60037F00229002CFE0B440
:1087B1007E0B12953612A80E60F17F0022E4900222
:1087C1000EF09002CFE0FF647E602C90020EE02458
:1087D10000F582E43400F583EFF090020EE004F03E
:1087E10012953690020EE0D3947840037F00221256
:1087F100A80E60CE7F00227B017A00790090020EE4
:10880100E024FEFD1296F190020EE0FE24FEF582B8
:10881100E434FFF583E0FF9002D4E06F60037F0052
:108821002274FF2EF582E434FFF583E0FF9002D33A
:10883100E06F60037F002290020EE024FEF0E090E2
:058841000100F07F01C1
:01884600220F
:108A2B00E49002CEF0120003120003E49002CFF0A8
:108A3B0030C10A30B3FA9002CE7401F02220C10A81
:108A4B0030B3FA9002CE7402F022A2C19215E490D8
:108A5B0002D0F090020FF012A97112A806A3E0B495
:108A6B00061690020FE004F0E0B4030C9002CE74F3
:108A7B0003F0E49002D0F022E49002D0F0C2162072
:108A8B0016D512A7FB20DF1C30B3079002CE74045F
:108A9B00F022A2C1301501B350EBA2C19215D21630
:108AAB00D2DF80E12016D812A8064480F0A3E004A0
:0B8ABB00F0E0B407CA9002CE7405F092
:018AC600228D
:10953600E490020FF090020FE0C39408506112A766
:10954600FB20DF2030B3079002CE7404F022A2C1C4
:10955600301501B3500AA2C19215D216D2DF80E1AE
:10956600C21680DD20161C9002CFE0FFC313F04424
:1095760080F0A3E004F0E0B407079002CE7405F093
:1095860022801412A9719002D0E0B40504E4F080A0
:0F959600A412A806E4A3F090020FE004F0809660
:0195A50022A3
:0E7BBB0090021EEBF0A3EAF0A3E9F0A3EDF0B8
:107BC900C2AC7F807E0112A88E900224EFF0C2C45D
:107BD900D2A7D2A4C2A6D2C5E49002D0F0900222C4
:107BE900F0900224E02401FFE433FE900222E0C376
:107BF9009FEE6480F87480985014E4A3F0127CA975
:107C0900E0C3942640F7900222E004F080D3E49088
:107C19000223F0900221E0FF900223E0C39F502449
:107C290090021EE0FBA3E0FAA3E0F9122E28FF124E
:107C3900996290021FE475F001122EF7900223E079
:107C490004F080CF9002D4E0FF1299629002D3E051
:107C5900FF129962E4900223F0127CA9E0C3940A0E
:107C690040F7D2C4C2A7C2A4D2A612A8157F817EAA
:107C79000112A88E900225EFF0D394004021E490E0
:107C89000223F0900225E0FF900223E0C39F500FEA
:0F7C99007F057E0012A701900223E004F080E433
:0D7CA800227F7E129962900223E004F022F8
:05996200900226EFF069
:10996700BF7E04D2148002C214E4900227F0900252
:1099770026E054017004B2C580269002D0E004F0BE
:109987002014047F0180027F009002D0E0B4050418
:109997007E0180027E00EE5F600A12A962B2C5E412
:1099A7009002D0F0900226E0FFC313F012A9629054
:0B99B7000227E004F0E0C3940840B376
:0199C2002282
:0FA96200E4F5D875F9FD75E908D2DE30DFFD2286
:0700030012A7FB30DFFD2214
:0FA97100E4F5D875F9FE75E980D2DE30DFFD22FE
:09AA6000C2A4D2C4C2A7D2A622EE
:05A26B0090020DEFF070
:10A27000602AE490020EF090020DE0FFA3E0C39F7D
:10A28000501AC2847F027E0012A701D2847F027E10
:0CA290000012A70190020EE004F080DB39
:01A29C00229F
:10544700000011892312329B462457AD653674BF7D
:105457008C489DC1AF5ABED3CA6CDBE5E97EF8F72D
:10546700108101083393221A56A5472C75B7643E5D
:105477009CC98D40BFDBAE52DAEDCB64F9FFE8760D
:105487002102308B02101399672676AF443455BD3D
:10549700AD4ABCC38E589FD1EB6EFAE7C87CD9F5ED
:1054A7003183200A1291031877A7662E54B5453C1D
:1054B700BDCBAC429ED98F50FBEFEA66D8FDC974CD
:1054C7004204538D6116709F042015A9273236BBFD
:1054D700CE4CDFC5ED5EFCD7886899E1AB7ABAF3AD
:1054E7005285430C7197601E14A1052837B3263ADD
:1054F700DECDCF44FDDFEC5698E98960BBFBAA728D
:105507006306728F4014519D252234AB063017B9BC
:10551700EF4EFEC7CC5CDDD5A96AB8E38A789BF16C
:105527007387620E5095411C35A3242A16B107389C
:10553700FFCFEE46DCDDCD54B9EBA8629AF98B704C
:1055470084089581A71AB693C22CD3A5E13EF0B77C
:10555700084019C92B523ADB4E645FED6D767CFF2C
:1055670094898500B79BA612D2ADC324F1BFE0365C
:1055770018C109483BD32A5A5EE54F6C7DF76C7E0C
:10558700A50AB48386189791E32EF2A7C03CD1B53C
:10559700294238CB0A501BD96F667EEF4C745DFDEC
:1055A700B58BA40296998710F3AFE226D0BDC1341C
:1055B70039C3284A1AD10B587FE76E6E5CF54D7CCC
:1055C700C60CD785E51EF497802891A1A33AB2B3FC
:1055D7004A445BCD695678DF0C601DE92F723EFBAC
:1055E700D68DC704F59FE41690A98120B3BBA232DC
:1055F7005AC54B4C79D7685E1CE10D683FF32E7A8C
:10560700E70EF687C41CD595A12AB0A3823893B1BB
:105617006B467ACF485459DD2D623CEB0E701FF96B
:10562700F78FE606D49DC514B1ABA02292B983309B
:105637007BC76A4E58D5495C3DE32C6A1EF10F784B
:0596F10090021EEDF0E7
:1096F60074FFA3F0A3F090021EE0D39400403F1243
:109706002E28FF90021FA3E06F25E0FFE433FE74CE
:10971600472FF58274543EF583E493FC740193FD60
:1097260090021FE0FFECFEED6FFFEEF0A3EFF0906E
:10973600021EE014F0740129F9E43AFA80B89002A6
:109746001FE0FEA3E0F4FFEEF4FCEF9002D4F0AECF
:0697560004EE9002D3F0C6
:01975C0022EA
:10A70100EF4E6019EF1FAC0670011E4C600FE4F5AF
:0EA71100D875F94CF5E9D2DE20DFE980FB2295
:10A7750057494445312000574944453220000D0AC8
:0CA78500444947492D3E5246203A20002E
:109FCA001FEF25E0FF74002EF582E43400F583EDDF
:109FDA0054E1F074002EF582E43400F58322EE7524
:109FEA00F007A414F0AF067BFF227B017A00790008
:0E9FFA00900100E0FD22F0900212E004F0223F
:10A8F70090000DE020E00B128E3FEF640160031221
:03A907008ECF22CE
:108E3F0090020F7403F07F857E0112A88EEF6401FC
:108E4F00707B90020FE0FED3940840037F002290C6
:108E5F000210129FE87AA7797512A045EF6401708E
:108E6F0043900210E0FE2400129FE0E0FD541EC369
:108E7F0013FF7002FF22129FCAE04FF0EF700D90A8
:108E8F000210E02400129FE0E04480F07F877E0113
:108E9F0012A88EBF010890020FE0FF127685129183
:108EAF00F47F0122900210E02400129FE0E030E0F6
:0F8EBF00037F002290020FE004F0028E517F002B
:018ECE002281
:108ECF0090020F7403F07F867E0112A88EEF64016B
:108EDF00707B90020FE0FED3940840037F00229036
:108EEF000210129FE87AA7797C12A045EF640170F7
:108EFF0043900210E0FE2400129FE0E0FD541EC3D9
:108F0F0013FF7002FF22129FCAE04FF0EF700D9017
:108F1F000210E02400129FE0E04480F07F877E0182
:108F2F0012A88EBF010890020FE0FF1276851291F2
:108F3F00F47F0122900210E02400129FE0E030E065
:0F8F4F00037F002290020FE004F0028EE17F000A
:018F5E0022F0
:10A04500EF1475F007A4900211F0122E2860282550
:10A05500E0FFE433FE900211E02400129FE0E06F80
:10A065007001EE60037F0022740129F9E43AFA9049
:09A075000211E004F080D37F0128
:01A07E0022BF
:05768500900211EFF07E
:10768A00900100E0D39478400302779EE4900215BB
:10769A00F0A3F0FFFE12A88EEF700302779EE4902B
:1076AA000215F0A3F0900212F0900215E0FEA3E09A
:1076BA00FF12A88EEF25E0900214F070037440F0D8
:1076CA00900214E0FF900212E02417F582E43402DB
:1076DA00F583EFF0900216E004F07006900215E0D0
:1076EA0004F012A001E0C3940640BE7F877E001218
:1076FA00A88EEF25E044E090021DF0900213E0040A
:10770A00F0900100E0FF900214F0900211E075F091
:10771A0007A424F8FEC3EF9E900213F0E49002122D
:10772A00F0900213E0FF900212E0C39F50229002F1
:10773A0014E0FF2400129FE0E0FE74072FF582E4B4
:10774A003400F583EEF0900214E01412A00080D108
:10775A00900211E01475F007A4900214F0E490026C
:10776A0012F0900212E0FFC39407502174172FF50C
:10777A0082E43402F583E0FF900214E02400129FB1
:10778A00E0EFF0900214E00412A00080D59001000E
:04779A00E02407F0F0
:01779E0022C8
:1091F4007F8A7E0112A88EBF010320C6FD7F897E6F
:109204000112A88EBF010330B3FD7F887E0112A82E
:109214008E900212EFF0D394004021E4900211F0FA
:10922400900212E0FF900211E0C39F500F7F057E71
:109234000012A701900211E004F080E4C2B5129F6D
:10924400F41296F1129FF4127BBB7B017A007980B1
:10925400125F917BFF7AA77983E4FD1270C87B01CA
:0B9264007A007980E4FD1270C8D2B5DA
:01926F0022DC
:0FA98000E4F5D875F9FF75E940D2DE30DFFD222E
:0FA98F00E4F5D875F9FF75E9A0D2DE30DFFD22BF
:10A84700D2A312A9807E08EFC313FFB392A312A964
:08A8570080DEF4C2A302A98017
:10A85F00D2A312A98F7E08EFC313FFB392A312A93D
:08A86F008FDEF4C2A302A98FE1
:09AA690090020DE0FF14F0EF2251
:109B8F0090020DEDF025E0F0EF24FE601604702634
:109B9F0012AA69600BB2B77F017E0012A70180F095
:109BAF00D2B72212AA69600BB2B67F017E0012A74C
:109BBF000180F0D2B62212AA696011B2B7B2B6B262
:109BCF00B4B2B57F017E0012A70180EAD2B6D2B738
:059BDF00D2B5D2B42252
:10A56F002056657273204E45542D3531544E43207D
:10A57F0032303134303331362000563A32303134C4
:05A58F003033313600FD
:10A16100900298E508F0A3E509F02290029AE50A29
:10A17100F0A3E50BF022900296E50CF0A3E50DF0BB
:10A1810022900294E50EF0A3E50FF02290029CE5E7
:07A1910010F0A3E511F0221C
:10A8770012975D12A95212AA3912A9FD12A79112B5
:07A88700983212A52380ECBA
:10A1CF0030803230812FE490020DF0C28000208168
:10A1DF0024D2800030811E7F017E0012A7019002E1
:10A1EF000DE004F0E0C3940A40E1125A23C2AFC25B
:05A1FF00B4C2B580FEB2
:01A204002237
:107F9D0012A2CEEF7010C2AFC2B4C2B5125A23D224
:107FAD00B5D2B475C7207F8012807E7F00FEC006DB
:107FBD00C0077F817E0012A88EEFFDD0E02DF50960
:107FCD00D0E03400F5087F827E0012A88EEF7F008E
:107FDD00FEC006C0077F8312807EFDD0E02DF50B1D
:107FED00D0E03400F50A7F00128074C006C007741B
:107FFD00010FFE12A88EEFFDD0E02DF50DD0E0346F
:10800D0000F50C7F02128074C006C0077F0312803A
:10801D0085FDD0E02DF50FD0E03400F50E7F8312F5
:10802D0080857004D2A58002C2A57F907E0112A822
:10803D008EEF7F00FEC006C0077F917E0112A88ED5
:10804D00EFFDD0E02DF511D0E03400F51012A16157
:10805D00C20812A16CC20912A177C20C12A182C270
:10806D000B12A18DC20A227E0112A88EEF7F00FE97
:0F807D00227E0012A88EEF227E0112A88EEF2223
:10975D0043B70243B80243B71012A1CF12AA60D289
:10976D00B475BBFF75B30475B404C2A312A6E3129E
:10977D00AA8612AA7BD2B7D2B612A9E3127F9D1286
:10978D00A9C812A9F012A9D6127EA6126D0A12A5A9
:10979D00B8126A45126A457D027F03129B8F7F01C5
:1097AD0012A26BC28C9001017414F0C28CC28D7523
:0C97BD008C4CE4F58AD28CD2A9D2AF22E9
:03000B00027CB5BF
:107CB500C0E0C0F0C083C082C0D075D000C000C095
:107CC50001C002C003C004C005C006C007C28CC203
:107CD5008D758C4C758A00D28C900101E014F0E012
:107CE5006003027D937414F0E5094508601A90025B
:107CF50099E024FFF0900298E034FFF0E07002A3D1
:107D0500E0700512A161D208E50B450A601A9002E0
:107D15009BE024FFF090029AE034FFF0E07002A3AC
:107D2500E0700512A16CD209E50D450C601A9002B0
:107D350097E024FFF0900296E034FFF0E07002A394
:107D4500E0700512A177D20CE50F450E601A90027E
:107D550095E024FFF0900294E034FFF0E07002A378
:107D6500E0700512A182D20BE5114510601A900250
:107D75009DE024FFF090029CE034FFF0E07002A348
:107D8500E0700512A18DD20A12A94112A6C5D0072D
:107D9500D006D005D004D003D002D001D000D0D079
:097DA500D082D083D0F0D0E0328E
:10731E00C0A80178FFFFFF00C0A801010008DC0132
:10732E00020392E5A2B674EC80DC92E5A2B6746517
:10733E0073740000003030300000002133313334DC
:10734E002E33314E2F31323032302E3232457220C2
:10735E003132330000000000000000000000000089
:10736E00000000000000000000000000000000000F
:10737E0000000000000000000000000000000000FF
:10738E0000000000000000000000000000000000EF
:10739E0000000000000000000000000000000000DF
:1073AE0000000000000000000000000000000000CF
:1073BE0000000000000000000000003D33343437B0
:1073CE002E30304E2F31313334332E3730455F630C
:1073DE00303030733030306730303074303839728E
:1073EE0030303070303030683436623130303130D9
:1073FE002057585F62656163656E000000000000F3
:10740E00000000000000000000000000000000006E
:10741E00000000000000000000000000000000005E
:10742E00000000000000000000000000000000004E
:0B743E00000000000000000000000043
:10A4FC0090021EE0FEA3E0FFE4FD12A5E3E004F0F1
:10A50C002275C65A75C6A52290021EE004F022ECF4
:07A51C00F5C3AF058FC42257
:10A2CE007F1C12A2F660037F00227F1D12A2F6648D
:10A2DE000860037F00227F1E7E0012A88EEF64DCD2
:0FA2EE0060037F00227F01227E0012A88EEF22E4
:0EA9BA00E4F5C7F5C5F5C675C3FF75C4FF22E9
:04A88E00AD07AC0660
:10A8920075C78275C50112A51B12A50D00AFC212A4
:02A8A200A9BA51
:01A8A4002291
:10A90A00AD07AC0612A51B75C78275C50312A50D46
:03A91A0002A9BAD5
:10A35800AD07AC0675C78275C50212A51B122E285B
:10A36800F5C212A50D000DBD00010C740129F9E418
:0DA378003AFA900225E014F070E002A9BA54
:07A5DC007F8412A5E37F85D7
:10A5E300AB07AA0675C78275C502EAF5C3AF038F29
:0CA5F300C4AF058FC212A50D0002A9BA6A
:105A2300E4FFFE12A90A7BFF7A73793C9002257486
:105A330007F0E4FF12A3587D0A7F0712A5E37BFF5B
:105A43007A7379439002257407F07F0912A3587A79
:105A530073791E9002257412F07F1012A3587A7383
:105A63007930900225740CF07F2212A358E4FD7F55
:105A73002E12A5E37F2F12A5E37F3012A5E30D7F3E
:105A83003112A5E31D7F3212A5E37F3312A5E37F15
:105A93003412A5E37F4012A5E37F8012A5E37D784E
:105AA3007F8112A5E37D027F8212A5E37D587F8368
:105AB30012A5E37D0112A5DC7D0A7F8712A5E39081
:105AC300021EE4F0A37490F0E4FCEC90734993FDA0
:105AD300601390021EE0FEA3E0FF12A506700312FE
:105AE300A5140C80E512A4FC700312A514E4FDFFB9
:105AF3007E0112A5E3E404FF12A5E37F0212A5E3EE
:105B03007F0312A5E37F0412A5E30D7F0512A5E32E
:105B13007D0D7F0712A5E3E4FD7F0812A5E37F0B4C
:105B230012A5E390021E7401F0A37410F0E4FCECE0
:105B33009073C993FD601390021EE0FEA3E0FF1271
:105B4300A506700312A5140C80E512A4FC700312C1
:105B5300A5147D017F807E0112A5E31D7F8112A51F
:105B6300E37F8312A5E312A5DC7F8612A5E37F877B
:105B730012A5E30D7F8812A5E31D7F8912A5E37F9C
:105B83008A12A5E37F8B12A5E37F8C12A5E37F8D99
:105B930012A5E37F8E12A5E37F9012A5E37F9112F6
:105BA300A5E37F9212A5E37D097F9312A5E3E4FDAC
:105BB3007F9412A5E37D217F9512A5E37D2F7F9628
:105BC30012A5E37D237F9712A5E3E4FD7F9812A539
:105BD300E37F9912A5E37F9A12A5E37D0B7F9B12C6
:105BE300A5E37D017F9C12A5E37D1D7F9D12A5E3A7
:075BF300E4FD7FB002A5E311
:0CAA1500424C2D3E52462F49533A20007F
:10A71F0074862FF582E43401F583227B017A007968
:0EA72F0080227B017A007900900100E0FD227B
:0EA9C800759850758921758DFDD28E02A815E7
:10A81500C2ACC217E4900206F0FF12A71FE4F00FC6
:09A825000FEFC3948040F3D2ACA4
:01A82E002207
:030023000297C978
:1097C900C0E0C083C082C0D0309906C299D2188047
:1097D9004F30984CC298301707900206E4F0804049
:1097E900900206E0248612A722E599F0900206E08D
:1097F90004F0E599B4C01CE0D3940E40169001869C
:10980900E0B4C008A3E07004D2178014C217900214
:1098190006E4F0900206E0D3947E4004C217E4F017
:09982900D0D0D082D083D0E0320F
:1098320030B364301761C2B5E4900100F07F02904A
:109842000206E014FEEFC39E501A12A71FE0FE7438
:10985200FE2FF582E434FFF583EEF0900100E00480
:10986200F00F80DB12A7311296F112A731127BBBE7
:1098720012A72A125F9112A72A12779F12A72A1201
:1098820068DB7BFF7AAA7915E4FD1270C812A72A59
:07989200E4FD1270C8D2B51D
:0198990022AC
:0AAA4300C2188F993018FDC21822C6
:109174000D0A4750532D3E4750524D43203A20206C
:10918400494F312020475053204E4F20636F6E6E5D
:10919400656374210D0A000D0A4750532D3E475054
:1091A400524D43203A20000D0A4750532D3E47505C
:1091B400524D43203A2020475053204E4F204C4FCD
:1091C400434B210D0A004750532D3E4750524D4307
:1091D400203A20004750532D3E4750474741203AFC
:1091E4002000244750524D43002447504747410034
:10614300E0FAA3E0FB7C037DE8FFAE02122EA2EF90
:106153002430FF900227E02474F582E43402F583AF
:10616300EFF0900227E004F07C007D64AF03AE0201
:10617300122EA27C007D0A122EA2ED2430FFE02411
:1061830074F582E43402F583EFF0900227E004F023
:1061930022900218E0FBA3E0FAA3E0F974742EF551
:1061A30082E43402F583EDF00E0F8F8275830012C3
:1061B3002E41FD74742EF582E43402F583EDF00E66
:1061C3000F8F82758300122E41FD74742EF582E4C5
:1061D3003402F58322900218E0FBA3E0FAA3E0F96E
:1061E3008F82758300022E41EF2BFBEE3AFA7D0A74
:1061F3007C00E024D0FFE434FFFE022E9090020ED8
:10620300E0FBA3E0FAA3E0F922EF2BFFEE3AFEA3B3
:10621300E090021D24D0FDEC34FFCD2FFFED3EF0C6
:10622300A3EFF022AA06AB077C037DE8E024D0FFAE
:10623300E434FFFE022E90A3F07B017A017903225E
:10624300E0FAA3E0FB7C007D0AFFAE02122EA27CE3
:10625300007D0A122EA2ED2430FF90022722EBF0DC
:10626300A3EAF0A3E9F022E024D075F00AA4FF2208
:1062730074112DF582E43402F583EFF00C0D2290B6
:10628300021FE0FEA3E0FF22900221E0FEA3E0FF55
:1062930022900227E024742224D075F064A42FFFF7
:1062A300E024D02F22EF75F00A84E5F022E0FCA36E
:1062B300E0FDC39FEC9E22ED9FFFEC9EF0A3EFF069
:0B62C30022E0FF75F00A842430FE2268
:059D1F00900218EFF0B6
:109D2400E4F5AF9001847403F07F8C7E0112A88E59
:109D3400EF7005759CFA8003759CFD43A210900298
:109D440018E024FF9210C20FE4900185F0FF740321
:109D54002FF582E43401F583E4F00F0FEFC3948010
:059D640040EC75AF01A9
:019D690022D7
:10A3B0007F927E0112A88E900289EFF024FE600E3B
:10A3C00014600E24027013300A10C20A800902863B
:0BA3D000F812A5FFBF0103128F5F22EF
:10A5FF003092037F00227F017E0012A70130920369
:10A60F007F00223092FD7F017E0012A7013092F36E
:03A61F007F012296
:1099C300E4FF129D1FE4900217F0200F1E7F017E1B
:1099D3000012A701900217E004F0E0D3942840EAB4
:1099E300E4F5AF7BFF7A917974802EE4F5AF7BFFCA
:1099F3007A91799BFD1270C812623CE4FD1270C823
:109A030012623C12A483BF010912623C12898C7F4B
:109A130001227BFF7A9179ABE4FD1270C87F0022AB
:108F5F00E4FF129D1FE490020DF0200F07128FD730
:108F6F0040F880407BFF7A9179CAE4FD1270C812F5
:108F7F00623CE4FD1270C812623C12A483BF011060
:108F8F0012623C12898C12623C127DAED20D8002AD
:108F9F00C20D7F01129D1FE490020DF0200F0912E8
:108FAF008FD740F8E4F5AF227BFF7A9179D8E4FDB3
:108FBF001270C812623CE4FD1270C812623C127843
:078FCF00AD300D0312808C90
:108FD600227F017E0012A70190020DE004F0E0D38B
:038FE600942822AA
:1086F800900270E01460161460552402600302872B
:108708009BE4F5AF90027004F0E4FF803F200F0374
:108718000287A07BFF7A9179CAE4FD1270C81262C1
:108728003CE4FD1270C812623C12A483BF0110120F
:10873800623C12898C12623C127DAED20D8002C25C
:108748000DE4F5AF9002707402F07F01029D1F30B6
:108758000F467BFF7A9179D8E4FD1270C812623C0B
:10876800E4FD1270C812623C1278AD300E1090020F
:1087780073E004F0E0D394054019C20E8015300D63
:1087880012128581BF010A12808CD20EE490027306
:09879800F08000E4900270F02270
:109C3800900103E064246007E4900185F0FF22208E
:109C4800101D90020A74FFF0A37491F074E612627A
:109C58003A12A07FBF0105D20FE4F5AF7F00229032
:109C6800020A74FFF0A37491F074ED12623A12A024
:0F9C78007FBF0108D20FE4F5AF7F01227F0022EA
:10A5B800E4900287F0A3F090025CF090025AF090C9
:10A5C8000272F0900271F0C20D900273F0C20E9008
:04A5D8000270F022FB
:0678AD0090020E12626160
:1078B300E4FFFE90020E1261DBFD6009B42C010EA1
:1078C3000FEEB409EE90020E1261DBB42D0C7F06AD
:1078D3009002547430F0A3DFFC22E4FE90020E12F7
:1078E30061DBFD642E601074112EF582E43402F521
:1078F30083EDF00E0F80E57F069002547430F0A301
:10790300DFFCEE24FE601314601E14603014604A22
:107913002404706B9002110279AD900211E0900281
:1079230058F09002120279AD900211E0900257F0E4
:10793300900212E0900258F0900213806D900211B1
:10794300E0900256F0900212E0900257F09002137A
:10795300E0900258F09002148050900211E09002DF
:1079630055F0900212E0900256F0900213E090025C
:1079730057F0900214E0900258F0900215802B907B
:107983000211E0900254F0900212E0900255F09040
:107993000213E0900256F0900214E0900257F09028
:0F79A3000215E0900258F0900216E0900259F0A1
:0179B20022B2
:06A4830090021812626154
:10A48900E4FFFE9002181261DB6009B42C010E0F83
:10A49900EEB402EF9002181261DBB441037F01228E
:02A4A9007F0032
:01A4AB00228E
:06898C0090021812626166
:10899200E4FFFE1261D86009B42C010E0FEEB4039D
:1089A200F2E4FE1261D8FD642E60091261CDEDF091
:1089B2000E0F80EF126194EDF00E0F1261D8642C4D
:1089C20060030F80F60F9002181262031261C4ED69
:1089D200F00E0F1261CD742FF00E1261D8642C606C
:1089E200030F80F60F1261D8FD642E60091261CD6B
:1089F200EDF00E0F80EF126194EDF00E0F1261D8C0
:108A0200642C60030F80F60F900218126203126149
:108A1200C4EDF00E1261CDE4F07F997E0112A88EB2
:088A2200BF010312423D7F0178
:018A2A002229
:10423D0090027412626AA3E024D02F900223F090B2
:10424D0002777D641261F3900276126227900279F3
:10425D001261EBEF2BFFEE3AFEA3E090021B126210
:10426D001790027BE0900225F0E4900227F0126295
:10427D00941261D0E0642F600512618D80F012619F
:10428D008DE4FF1262941261D0E0642E600612611B
:10429D008D0F80EFEF24FB603504707590027D1259
:1042AD00626AA3E024D02F900224F09002807C005B
:1042BD007D6412622FAA06AB0790027F12622B90CB
:1042CD0002821261EB12620C900284024319900279
:1042DD007E12626A90027DE090027F12629B9002D4
:1042ED0024F0900281E024D0FFE434FFFE7C007DB9
:1042FD0064122E90900280126227EF2BFBEE3AFA99
:10430D009002831261F112620C900285E0900226F8
:10431D00F07F9B7E0112A88E90021FE4F0A3EFF0B8
:10432D007F9A7E0112A88EBF013012628290021C0C
:10433D00E02FF090021BE03EF0C3A3E094709002DA
:10434D001BE09417404BA3E02490F090021BE03447
:10435D00E8F0900223E004F0803712628290021B95
:10436D001262B0400890021B1262BA802490021CA7
:10437D00E02470F090021BE03417F0126282C390BB
:10438D00021CE09FF090021BE09EF0900223E014CF
:10439D00F07F9D7E0112A88E900221E4F0A3EFF034
:1043AD007F9C7E0112A88EBF013012628B90021E7F
:1043BD00E02FF090021DE03EF0C3A3E09470900258
:1043CD001DE09417404BA3E02490F090021DE034C3
:1043DD00E8F0900224E004F0803712628B90021D09
:1043ED001262B0400890021D1262BA802490021E23
:1043FD00E02470F090021DE03417F012628BC39030
:10440D00021EE09FF090021DE09EF0900224E01449
:10441D00F0E4900227F09002231262C4126294120B
:10442D0061D0EE12618C1262A812617E90021B1295
:10443D006143E024741261D0742E12618C90021BC2
:10444D001262431261817C007D0AAF03AE021261DC
:10445D007A900225E0FF9002271261817F067E008F
:10446D0012A88E900227126181900224E0FFD3944E
:10447D00634020E0FE75F064842430FD12629412D6
:10448D0061D0ED12618CEE75F00A841262A92430B0
:10449D00FE80099002241262C4900227E024741257
:1044AD0061D0EE12618C1262A812617E90021D1213
:1044BD006143E024741261D0742E12618C90021D40
:1044CD001262431261817C007D0AAF03AE0212615C
:1044DD007A900226E0FFA3126181E024741261D06C
:0444ED00E412618CE8
:0144F10022A8
:1085810090025BE0F97002FF22900287E0FEA3E017
:10859100FF900252E0FAA3E0FBD39FEA9E4008EB72
:1085A1009FFDEA9EFC8015900252E0FEA3E0FFC30E
:1085B100900288E09FFD900287E09EFCD3ED94B489
:1085C100EC9400401074689D90020EF074019C9030
:1085D100020DF0800890020DECF0A3EDF0D39002B3
:1085E1000EE0941990020DE094004006E4900271AF
:1085F100803A900271E004F0E9C3940A500CE0C3A0
:1086010094324003E480257F002290025BE0C39412
:1086110032500F900271E0C3941E4003E4800D7F3D
:108621000022900271E0C394144014E4F0900252CD
:10863100E0FFA3E0900287CFF0A3EFF07F01227F5C
:018641000038
:018642002215
:067DAE0090020E1262615A
:107DB400E4FCFD1262008C821261E56009B42C01BE
:107DC4000D0CEDB407ED1262008C821261E5B42C47
:107DD40003E48041E4FD1262008C821261E5FF64D9
:107DE4002E600512627380EEED24FD601004701F96
:107DF40090021112626AA3E024D02F80189002121C
:107E040012626A900211E090021312629B80069043
:107E14000211E024D090025BF01262008C821261A5
:107E2400E5642C60030C80F10C1262008C821261F8
:107E3400E5B42C08E4900252F0A3F022E4FD1262AF
:107E4400008C821261E5FF642E600512627380EE7D
:107E5400ED24FD600C0470389002111261F1A380CE
:107E64001B9002121261F1AA06AB079002117D6405
:107E74001261F5EF2BFFEE3AFE900213E024D0FDE1
:107E8400EC34FFCD2FFFED3E900252F0A3EFF02231
:107E9400900211E024D0FEE434FF900252F0A3CE0D
:017EA400F0ED
:017EA50022BA
:10A07F0090020712626190020A126203122E28FFE9
:10A08F006025900207126203122E286F60037F0073
:10A09F0022900208E475F001122EF790020BE4757E
:0AA0AF00F001122EF780CF7F01228E
:10A66600A3E02403F582E43401F583E59BF0900131
:10A6760085E004F022E02403F582E43401F583E466
:02A68600F022C0
:03004300028AC767
:108AC700C0E0C0F0C083C082C0D075D000C000C075
:108AD70001C002C003C004C005C006C007E59A3044
:108AE700E106539AFD028B42E59A30E04E539AFE17
:108AF700900184E06401701512A666E59BB40A0B29
:108B070012A67B12A67412A4D5802B802490018410
:108B1700E06403702112A666900102E004F0E59B71
:108B2700B40A0E90018512A67B12A674129C388097
:108B37000512AA218005900185E4F0D007D006D060
:108B470005D004D003D002D001D000D0D0D082D03D
:068B570083D0F0D0E032F3
:0CAA2100900185E0D3947E4002E4F02216
:0DA9F00043A210759A50758E10759CF422CC
:10004600000000000000000000000C079409D430F6
:1000560054304C202020202020202020200020006A
:1000660020002000200020002000200060204010FA
:100076004010C018800F00070000000000000000BC
:10008600000000000000000000001800240024000A
:1000960024002400140018000000000000000000E6
:1000A600000000000000000000000000000000004A
:1000B600000000000000000000000000000000003A
:1000C600000000000000000000000000000000002A
:1000D600000000000000000000000000000000001A
:1000E600000000000000000000000000000000000A
:1000F60000000000000000000000000000000000FA
:100106000000000000000000C003C003C003C001DF
:10011600C001C001C001C001C00180018001800191
:100126008001800180018001800100000000000044
:10013600C003C003C00380010000000000000000EF
:1001460000000000000000000000700E700E700E2F
:10015600700E300630063006000000000000000079
:100166000000000000000000000000000000000089
:100176000000000000000000000000000000000079
:100186000000000000000000000000006018601879
:100196006018601860183018FE7FFE7F300C300C37
:1001A600300C300C180CFE7FFE7FFE7F18061806FA
:1001B600180618060C0600000000000000000000EB
:1001C600000000000000800180018001E007F80FB8
:1001D600B81D9C1D9C199C199C01B801F801F001E1
:1001E600C007800F801F801D9C399C399C399C1943
:1001F6009C1DF81FF00FC0038001800180010000E4
:100206000000000000000000000000003C103E1846
:100216006608660C660466046602660266013E01AE
:100226009C08803CC03640664066206620661066A4
:1002360010660836083C08080000000000000000B0
:10024600000000000000000000000000E003F007CE
:1002560038061806180618063807B003F001F0002D
:100266007800FC00CC31CE318633063F061E0E1CCC
:100276001E7EFC7FF863E000000000000000000026
:10028600000000000000000000000000C000C000E8
:10029600C000C000C000C000000000000000000058
:1002A6000000000000000000000000000000000048
:1002B6000000000000000000000000000000000038
:1002C6000000000000000020007000380018000C3C
:1002D6000006000600030003000300018001800100
:1002E60080018001800180010003000300030006F5
:1002F6000006000C001C0018003000200000000062
:1003060000000000000004000E000C001800300081
:10031600300060006000C000C000C000C000C00027
:10032600C000C000C000C000C000C0006000600087
:100336007000300018001C000E00060000000000CF
:1003460000000000000000000000000080018001A5
:10035600800186619E79FC3FF00FC003F00FFC3FE1
:100366009E79866180018001800180010000000085
:100376000000000000000000000000000000000077
:100386000000000000000000000000000000000067
:100396000000800180018001800180018001FE7FD4
:1003A600FE7F800180018001800180018001800143
:1003B6000000000000000000000000000000000037
:1003C6000000000000000000000000000000000027
:1003D6000000000000000000000000000000000017
:1003E6000000000000000000000000000000000007
:1003F60038003C007C0038003000300018000C004B
:1004060000000000000000000000000000000000E6
:100416000000000000000000000000000000FE7F59
:10042600FE7F000000000000000000000000000049
:1004360000000000000000000000000000000000B6
:1004460000000000000000000000000000000000A6
:100456000000000000000000000000000000000096
:100466000000000000000000000000000000000086
:1004760018003C003C0018000000000000000000CE
:1004860000000000000000000000006000200030B6
:1004960000100018000C0004000600020003000112
:1004A6008001C000C000600020003000100018006D
:1004B60008000C0006000600020000000000000014
:1004C600000000000000000000000000E007F00F40
:1004D600381C1C1C1C380C380E300E300E300E30FA
:1004E6000E300E300E300E300E300C381C381C1804
:1004F600381CF80FE0078001000000000000000033
:1005060000000000000000000000000080038003DF
:10051600C003E003B80398038803800380038003C5
:1005260080038003800380038003800380038003AD
:10053600800380038003000000000000000000002C
:10054600000000000000000000000000F007F81F97
:100556003C1C1C380E38003800380018001C001CE3
:10056600000E000700038003C001E00070003800A1
:100576003C00FC3FFC3F00000000000000000000C3
:10058600000000000000000000000000E007F01F6F
:10059600381C1C380C38083800380018001EC007F4
:1005A600C00F001E00380038003808300E381C38DE
:1005B6003C1CF81FF007800100000000000000004E
:1005C600000000000000000000000000000C000E0B
:1005D600000E000F800F800DC00DE00C700C300C6B
:1005E600380C1C0C0C0C0E0CFF7FFF7FFF7F000CE1
:1005F600000C000C000C00000000000000000000D1
:10060600000000000000000000000000F81FF81FB6
:100616001800180018001C000C00EC03FC0F1E1E2E
:100626000E1C0038003800300030043806380E380A
:100636000E1EFC0FF807E00100000000000000009D
:100646000000000000000000000000000007000796
:100656008003C001C001E00070007000F80FF81FB1
:100666003C381C700E700E700E700E700E701C7082
:100676003C38F81FF00F8003000000000000000067
:10068600000000000000000000000000FE7FFE7F6A
:10069600007000380018001C000C000E0006000751
:1006A6000003800380038001C001C001C000E00098
:1006B600E000600070000000000000000000000084
:1006C600000000000000000000000000F007F80F26
:1006D6001C1C0C380C380C380C381C1C3C1EF00743
:1006E600F80F3C1E1E380E38063006300E300E3817
:1006F6001E3CFC1FF80FC0010000000000000000B7
:10070600000000000000000000000000F007F80FE5
:100716003C1E0E3C0E3806380638063806380E1CC7
:100726001E1EFC1FF80F0007000780038003C00190
:10073600C001E00060007000000000000000000042
:1007460000000000000000000000000000000000A3
:100756000000000000000000000000000000C001D2
:10076600C001C00100000000000000000000000001
:10077600C001C001C001C000000000000000000070
:100786000000000000000000000000000000000063
:100796000000000000000000000000000000C00192
:1007A600C001C001000000000000000000000000C1
:1007B600C001C001C003C00180018001C00060000B
:1007C600000000000000000000000020007000385B
:1007D600001C000600038001C000600038001C00F9
:1007E6000E000C0018007000E000C0018003000736
:1007F600000C00180030002000000000000000007F
:1008060000000000000000000000000000000000E2
:10081600000000000000FE7FFE7FFE7F000000005B
:10082600000000000000FE7FFE7F000000000000C8
:1008360000000000000000000000000000000000B2
:100846000000000000000000000004000E001C0074
:1008560038007000E000C00100030006000C00181C
:1008660000300038001C000E00078001C000600048
:1008760030001C000E000400000000000000000014
:10088600000000000000000000000000E007F80F74
:10089600381E1C1C1C381C381C1C001C001E000F9B
:1008A60080078003C001C001C001000000000000F5
:1008B600C001C001C001800000000000000000006F
:1008C600000000000000000000000000C007301813
:1008D60018100C20842BC66F624C624C324632468E
:1008E60032463246326632223223F21FE60C0400CA
:1008F6000C001818700680010000000000000000BF
:10090600000000000000000000000000C001C0035D
:10091600C003C003E003E00760077006700E700EA8
:10092600300C381CF81FF81FFC1F1C381C380E38FA
:100936000E700E700E700000000000000000000037
:10094600000000000000000000000000FE07FE0F8F
:100956000E1E0E380E380E380E380E380E1CFE0FD0
:10096600FE0F0E1E0E380E700E700E700E700E38C4
:100976000E3CFE1FFE0F00000000000000000000FD
:10098600000000000000000000000000E007F01F6B
:10099600783C38381C301C701C700E700E000E002F
:1009A6000E000E000E000E700E701C701C301C38EF
:1009B600383CF01FE00F800300000000000000003C
:1009C600000000000000000000000000FE01FE071D
:1009D6008E0F0E1E0E3C0E380E380E380E700E7030
:1009E6000E700E700E700E380E380E380E380E1C45
:1009F6000E1FFE0FFE0300000000000000000000B6
:100A0600000000000000000000000000FC3FFC3F6A
:100A16001C001C001C001C001C001C001C00FC1FF1
:100A2600FC1F1C001C001C001C001C001C001C00E1
:100A36001C00FC7FFC7F000000000000000000009E
:100A4600000000000000000000000000FE7FFE7FA6
:100A56000E000E000E000E000E000E000E00FE0F21
:100A6600FE0FFE0F0E000E000E000E000E000E0012
:100A76000E000E000E000000000000000000000046
:100A8600000000000000000000000000E007F00F7A
:100A9600781C38381C381C380C380E000E000E0036
:100AA6000E000E3F0E3F0E300E301C301C301C3830
:100AB600383CF83FE03780310000000000000000BD
:100AC6000000000000000000000000000E380E3894
:100AD6000E380E380E380E380E380E380E38FE3FE9
:100AE600FE3F0E380E380E380E380E380E380E38D9
:100AF6000E380E380E38000000000000000000001E
:100B0600000000000000000000000000C001C0015D
:100B1600C001C001C001C001C001C001C001C001C7
:100B2600C001C001C001C001C001C001C001C001B7
:100B3600C001C001C001000000000000000000006C
:100B4600000000000000000000000000003800382F
:100B560000380038003800380038003800380038CF
:100B66000038003800381C381C381C381C381C3833
:100B76003C1CF81FF00FC001000000000000000040
:100B86000000000000000000000000000E380E3CCF
:100B96000E1E0E0E0E078E03CE03CE01EE00FE01D4
:100BA600FE01BE039E030E070E070E0E0E1E0E1C42
:100BB6000E3C0E380E700000000000000000000021
:100BC6000000000000000000000000000E000E0003
:100BD6000E000E000E000E000E000E000E000E009F
:100BE6000E000E000E000E000E000E000E000E008F
:100BF6000E00FE7FFE7F00000000000000000000E7
:100C06000000000000000000000000001E781E7CAE
:100C16001E7C3E7C3E7C3E7C3E7E3E7E7E766E76B6
:100C26006E766E766E77EE73CE73CE73CE73CE73AC
:100C3600CE718E718E710000000000000000000071
:100C46000000000000000000000000001E381E38F2
:100C56001E383E383E387E386E38EE38EE38CE399D
:100C6600CE398E398E3B0E3B0E3F0E3E0E3E0E3E6D
:100C76000E3C0E3C0E380000000000000000000094
:100C8600000000000000000000000000E007F80F70
:100C9600381E1C3C1C380E380E300E700E700E704E
:100CA6000E700E700E700E700E700E381C381C38DA
:100CB6003C1CF81FF00F800100000000000000003F
:100CC600000000000000000000000000FC07FC1F00
:100CD6001C3E1C381C701C701C701C701C701C3850
:100CE6001C3EFC1FFC071C001C001C001C001C00FA
:100CF6001C001C001C00000000000000000000009A
:100D0600000000000000000000000000E007F80FEF
:100D1600381E1C3C1C380E380E300E700E700E70CD
:100D26000E700E700E700E720E730E3F1C3E1C3E41
:100D36003C1CF81FF03F8019000000000000000076
:100D4600000000000000000000000000FE07FE1F7B
:100D56000E1E0E380E380E380E380E380E380E3E71
:100D6600FE1FFE070E070E070E0E0E0E0E1C0E1CA5
:100D76000E380E380E700000000000000000000063
:100D8600000000000000000000000000E007F80F6F
:100D96003C1E1C1C1C381C381C003C007800F00350
:100DA600E007001F003E003800380E300E301E38B7
:100DB6001C3CF81FF00FC0010000000000000000FE
:100DC600000000000000000000000000FE3FFE3FA3
:100DD600C001C001C001C001C001C001C001C00105
:100DE600C001C001C001C001C001C001C001C001F5
:100DF600C001C001C00100000000000000000000AA
:100E06000000000000000000000000000E380E3850
:100E16000E380E380E380E380E380E380E380E389C
:100E26000E380E380E380E380E380E380E381C387E
:100E36003C3CF81FF00FC00300000000000000005B
:100E460000000000000000000000000007700E70A7
:100E56000E700E380C381C381C181C1C381C381C1C
:100E6600380E300E700E700670076007E003E00360
:100E7600C003C003C001C001000000000000000064
:100E8600000000000000000000000000C761C771FC
:100E9600C771C673C673C673EE736E336E336E3325
:100EA6006E366C3E6C3E6C3E3C3E3C1E3C1E3C1C14
:100EB6003C1C381C381C181C0000000000000000F8
:100EC6000000000000000000000000000E381C3882
:100ED6001C1C381C380E700E7007E003C003C001DE
:100EE600C001C003E00360077006300E380C181C02
:100EF6001C180E380E7000000000000000000000F4
:100F06000000000000000000000000000E700E301F
:100F16001C381C18381C380C300E70066007E003AD
:100F2600C003C001C001C001C001C001C001C001B1
:100F3600C001C001C0010000000000000000000068
:100F4600000000000000000000000000FC3FFC3F25
:100F560000380018001C000E000E00070003800376
:100F6600C001C001E00070007000380038001C00AD
:100F76000E00FE7FFE7F0000000000000000000063
:100F8600000000000000C03FC03FC000C000C0001D
:100F9600C000C000C000C000C000C000C000C0004B
:100FA600C000C000C000C000C000C000C000C0003B
:100FB600C000C000C000C000C000C03FC03F00006D
:100FC600000000000000000000000C000C001800EB
:100FD6001800180030003000600060006000C0009B
:100FE600C0008001800180010003000300060006A6
:100FF6000006000C000C0018001800180030000055
:10100600000000000000FE01FE0180018001800159
:1010160080018001800180018001800180018001C2
:1010260080018001800180018001800180018001B2
:1010360080018001800180018001FE01FE01000027
:1010460000000000C001E0037007380E181C000005
:10105600000000000000000000000000000000008A
:10106600000000000000000000000000000000007A
:10107600000000000000000000000000000000006A
:10108600000000000000000000000000000000005A
:10109600000000000000000000000000000000004A
:1010A600000000000000000000000000000000003A
:1010B6000000000000000000000000000000FFFF2C
:1010C60000000000F000E001C001800300030006FC
:1010D600000000000000000000000000000000000A
:1010E60000000000000000000000000000000000FA
:1010F60000000000000000000000000000000000EA
:1011060000000000000000000000000000000000D9
:1011160000000000000000000000E003F00F781E51
:101126001C181C18001CE01FF81B1C180C180E1CA1
:101136000E1EFC1FF83B60000000000000000000CF
:101146000000000000000000000000000E000E007D
:101156000E000E000E000E000E00CE07EE0F3E1E15
:101166001E1C1E380E380E380E380E380E381E3835
:101176001E1CFE1FEE0F8001000000000000000094
:101186000000000000000000000000000000000059
:1011960000000000000000000000C003F00F781EF1
:1011A6001C380C380E000E000E000E000E381C38CF
:1011B6001C3CF81FF00F800100000000000000003A
:1011C60000000000000000000000000000380038A9
:1011D60000380038003800380038E039F83F3C3E27
:1011E6001C3C0E380E380E380E380E380E380C38B9
:1011F6001C3CF83FF03BC00000000000000000006F
:1012060000000000000000000000000000000000D8
:1012160000000000000000000000C003F00F381EB0
:101226001C380C38FE3FFE3F0E000E000E001C3828
:101236001C38F81FF00F80030000000000000000BB
:10124600000000000000000000000000003F803F9A
:10125600C021C000C000C000C000FE1FFE1FC000AD
:10126600C000C000C000C000C000C000C000C00078
:10127600C000C000C0000000000000000000000028
:101286000000000000000000000000000000000058
:1012960000000000000000000000E071F07F380E42
:1012A600180C1C0C1C0C180C380EF007EC010C006A
:1012B6003C00F81FF83F0C300E300E38FC1FF007CC
:1012C6000000000000000000000000000C000C0000
:1012D6000C000C000C000C000C008C0FCC1F6C3C9E
:1012E6003C381C381C380C380C380C380C380C3888
:1012F6000C380C380C38000000000000000000001C
:101306000000000000000000000000008001C00393
:10131600C0010000000000000000C001C001C001C3
:10132600C001C001C001C001C001C001C001C001AF
:10133600C001C001C0010000000000000000000064
:10134600000000000000000000000000000E000E7B
:10135600000E0000000000000000000E000E000E4F
:10136600000E000E000E000E000E000E000E000E07
:10137600000E000E000E000600060807F803F8012E
:101386000000000000000000000000000C000C003F
:101396000C000C000C000C000C000C3C0C1E0C0F7E
:1013A6008C07CC03EC01FC033C031C070C0E0C0E53
:1013B6000C1C0C180C380000000000000000000097
:1013C6000000000000000000000000008001800115
:1013D60080018001800180018001800180018001FF
:1013E60080018001800180018001800180018001EF
:1013F6008001800180010000000000000000000064
:1014060000000000000000000000000000000000D6
:1014160000000000000000000000E738F77DFF7FB5
:101426008F6387618761876187618761876187616C
:1014360087618761876100000000000000000000EE
:101446000000000000000000000000000000000096
:10145600000000000000000000008C0FCC1F6C3C58
:101466003C381C381C380C380C380C380C380C3806
:101476000C380C380C38000000000000000000009A
:101486000000000000000000000000000000000056
:1014960000000000000000000000C003F00F781EEE
:1014A6001C3C0C380E300E700E700E700E301C3850
:1014B6003C3CF81FF00F8001000000000000000017
:1014C6000000000000000000000000000000000016
:1014D60000000000000000000000CE03EE0F7E1E9C
:1014E6001E1C1E380E380E380E380E380E381E38B2
:1014F6001E1CFE1FEE0FCE030E000E000E000E0089
:1015060000000000000000000000000000000000D5
:1015160000000000000000000000E039F83F7C3EBB
:101526001C3C0E380E380E380E380E380E380C3875
:101536001C3CF83FF03BE0390038003800380038F2
:101546000000000000000000000000000000000095
:1015560000000000000000000000381C381FB81F03
:10156600F801780078003800380038003800380074
:1015760038003800380000000000000000000000BD
:101586000000000000000000000000000000000055
:1015960000000000000000000000E007F00F381C0B
:1015A6001C181C003800F803F00F001E00381C3809
:1015B6001C38F81FF00FC0030000000000000000F8
:1015C6000000000000000000000000000000000015
:1015D600E000E000E000E000E000FE1FFE1FE0008B
:1015E600E000E000E000E000E000E000E000E000F5
:1015F600E000C03F803F000E000000000000000039
:1016060000000000000000000000000000000000D4
:10161600000000000000000000000C380C380C38F8
:101626000C380C380C380C380C380C380C380C3C90
:101636001C3C3C3FF83BE0000000000000000000BE
:101646000000000000000000000000000000000094
:10165600000000000000000000000E300C381C38AE
:101666001C18181C380C380C300E700670076007F2
:10167600E003C003C003C00100000000000000003A
:101686000000000000000000000000000000000054
:1016960000000000000000000000C761C761C673BB
:1016A600C67346336E336E336C326C3E6C1E3C1E14
:1016B600381E381E380C380C0000000000000000F0
:1016C6000000000000000000000000000000000014
:1016D600000000000000000000001C381C1C381C24
:1016E600300E7007E003C003C001E0036007700E10
:1016F600380E1C1C1C380000000000000000000012
:1017060000000000000000000000000000000000D3
:10171600000000000000000000000E300E381C38EB
:101726001C18181C381C380C300E70067006600722
:10173600E003C003C003C001C001EC00FC007C0054
:101746000000000000000000000000000000000093
:1017560000000000000000000000FC1FFC1F001C31
:10176600000E000700078003C001E000700038008B
:101776001C00FC3FFC3F00000000000000000000D1
:10178600000000000000003C000E000600060006F7
:101796000006000600060006000600060006000712
:1017A6008003800700060006000600060006000605
:1017B60000060006000600060006003E003800008F
:1017C600800180018001800180018001800180010B
:1017D60080018001800180018001800180018001FB
:1017E60080018001800180018001800180018001EB
:1017F60080018001800180018001800180018001DB
:101806000000000000003C007000700070007000D6
:101816007000700070007000700070007000600052
:10182600E001E00160007000700070007000700060
:10183600700070007000700070003C001C0000001A
:1018460000007020F820FC338C3F041E000C0000C2
:101856000000000000000000000000000000000082
:101866000000000000000000000000000000000072
:101876000000000000000000000000000000000062
:10188600000000000000000000000000FE03060348
:1018960006030603060306030603060306030603FA
:1018A60006030603060306030603060306030603EA
:1018B60006030603FE03000000000000000000000F
:1018C6000000000000000000000000000000000012
:1018D600000000000000030000C0070000E0070051
:1018E60000E0070000300F0000300F0000181E0057
:1018F60000181E00000C3C00000C3C00000678009E
:10190600000678000007F80000FFFF008001F001E4
:101916008001E001C001E001C000C003E000C00397
:101926006000C00770008007FE03F07F0000000023
:1019360000000000000000000000000000000000A1
:101946000000000000000000000000000000000091
:101956000000000000000000FCFF7F00C003E0075D
:10196600C003800FC003001FC003003EC003003E3B
:10197600C003003EC003001FC003800FC003E00386
:10198600C0FF7F00C0030000C0030000C0030000CA
:10199600C0030000C0030000C0030000C003000035
:1019A600C0030000C0030000FC3F00000000000070
:1019B6000000000000000000000000000000000021
:1019C6000000000000000000000000000000000011
:1019D6000000000000000000FCFF7F00C003F007CD
:1019E600C003800FC003001FC003001FC003001FF9
:1019F600C003000FC003800FC003F003C0FF3F0009
:101A0600C0031F00C0031E00C0033C00C0037800D3
:101A1600C003F000C003F001C003E003C003C0032D
:101A2600C0038007C003000FFC3F00FE000000005B
:101A360000000000000000000000000000000000A0
:101A46000000000000000000000000000000000090
:101A5600000000000000000000FE0F02C003F003BB
:101A6600E0008003700000077800000678000000A0
:101A7600F8000000F00F0000C0FF000000FE1F008D
:101A860000E0FF000000FE030000F0070000C00FAA
:101A96000000000F0C00000F1800000F3800800730
:101AA6007800C003F003F00030FC1F0000000000C7
:101AB6000000000000000000000000000000000020
:101AC6000000000000000000000000000000000010
:101AD6000000000000000000000000000000000000
:101AE60000000000000000000000000000000000F0
:101AF60000000000000000000000000000000000E0
:101B060000000000000000000000000000000000CF
:101B160000000000000000000000000000000000BF
:101B260000000000000000000000000000000000AF
:101B3600000000000000000000000000000000009F
:101B4600000000000000000000000000000000008F
:101B5600000000000000000080FFFF0780FFFF0379
:101B6600800100008001000080010000C00100002B
:101B7600C0000000C0F03F00C00CF801C003E00345
:101B8600C000C0070000800F0000800F0000800F1B
:101B96000000800FE003800FF003C007F001C007CC
:101BA600E001E0038007F80000FC1F0000000000D1
:101BB600000000000000000000000000000000001F
:101BC600000000000000000000000000000000000F
:101BD60000000000000000000000030000C0030039
:101BE60080FF030000C0030000C0030000C0030024
:101BF60000C0030000C0030000C0030000C00300D3
:101C060000C0030000C0030000C0030000C00300C2
:101C160000C0030000C0030000C0030000C00300B2
:101C260000C0030000E0070080FFFF010000000085
:101C3600000000000000000000000000000000009E
:101C4600000000000000000000000000000000008E
:101C56000000000000000000F0FFFF0F70C0031E30
:101C660038C0031818C003100CC0033000C00300AE
:101C760000C0030000C0030000C0030000C0030052
:101C860000C0030000C0030000C0030000C0030042
:101C960000C0030000C0030000C0030000C0030032
:101CA60000C0030000C0030000FC3F00000000006D
:101CB600000000000000000000000000000000001E
:101CC600000000000000000000000000000000000E
:101CD6000000000000000000FE03C0FFE007000C4B
:101CE600E00F000C601F000C603E000C607C000CD6
:101CF60060F8000C60F0010C60E0030C60C0070C9B
:101D060060800F0C60001F0C60003E0C60007C0CB5
:101D16006000F00C6000E00D6000C00F6000800FF6
:101D26006000000F6000000EFE07000C00000000BF
:101D3600000000000000000000000000000000009D
:101D4600000000000000000000000000000000008D
:101D5600000000000000000000E07F0C003EC00F05
:101D6600800F001EC003001CE0010018F0000030C8
:101D7600F8000000780000007C0000007C000000F5
:101D86007C0000007C0000007C0000007C0000005D
:101D9600F8000000F8000030F0010010E003000C2D
:101DA600C0070006001FC00100F03F000000000051
:101DB600000000000000000000000000000000001D
:101DC600000000000000000000000000000000000D
:101DD6000000000808080808080800001818000095
:101DE60000486C2412000000000000000000000003
:101DF6000000002424247F1212127F121212000007
:101E06000000081C2A2A0A0C1828282A2A1C080856
:101E160000000022251515152A5854545422000096
:101E26000000000C1212120A76252911916E00008C
:101E36000006060403000000000000000000000089
:101E4600004020101008080808080810102040005C
:101E560000020408081010101010100808040200F0
:101E66000000000008086B1C1C6B0808000000003E
:101E760000000000080808087F080808080000009D
:101E86000000000000000000000000000606040339
:101E96000000000000000000FE000000000000003E
:101EA6000000000000000000000000000606000020
:101EB60000008040402020101008080404020200A0
:101EC60000000018244242424242424224180000C6
:101ED600000000080E08080808080808083E000068
:101EE6000000003C4242422020100804427E0000CE
:101EF6000000003C4242201820404042221C0000C4
:101F0600000000203028242422227E202078000091
:101F16000000007E0202021A26404042221C0000F7
:101F2600000000382402021A264242422418000009
:101F36000000007E22221010080808080808000089
:101F46000000003C4242422418244242423C000027
:101F5600000000182442424264584040241C0000FD
:101F6600000000000000181800000000181800000B
:101F7600000000000000000800000000000808043F
:101F86000000004020100804020408102040000051
:101F96000000000000007F0000007F00000000003D
:101FA600000000020408102040201008040200006F
:101FB6000000003C42424640201010001818000065
:101FC6000000001C225A555555552D42221C000072
:101FD6000000000808181414243C224242E70000BE
:101FE6000000001F2222221E22424242221F00001F
:101FF6000000007C4242010101010142221C000056
:102006000000001F2242424242424242221F00007A
:102016000000003F4212121E12120242423F00000E
:102026000000003F4212121E1212020202070000B6
:102036000000003C2222010101712122221C000025
:10204600000000E7424242427E42424242E700002E
:102056000000003E0808080808080808083E0000B6
:102066000000007C10101010101010101010110F2E
:102076000000007722120A0E0A12122222770000AE
:10208600000000070202020202020202427F000072
:1020960000000077363636362A2A2A2A2A6B0000AE
:1020A600000000E346464A4A525252626247000026
:1020B6000000001C2241414141414141221C0000D7
:1020C6000000003F424242423E0202020207000076
:1020D6000000001C2241414141414D53321C600029
:1020E6000000003F4242423E1212222242C7000036
:1020F6000000007C4242020418204042423E00009A
:102106000000007F4908080808080808081C0000A5
:10211600000000E74242424242424242423C000044
:10212600000000E742422224241414180808000084
:102136000000006B494949495555362222220000C4
:10214600000000E7422424181818242442E700005F
:10215600000000772222141408080808081C000052
:102166000000007E2120101008040442423F0000B7
:102176000078080808080808080808080808780009
:102186000000020204040808081010202020404025
:10219600001E1010101010101010101010101E003D
:1021A60000384400000000000000000000000000AD
:1021B600000000000000000000000000000000FF1A
:1021C60000060800000000000000000000000000FB
:1021D600000000000000003C4278444242FC00003F
:1021E600000000030202021A26424242261A00009A
:1021F60000000000000000384402020244380000DB
:1022060000000060404040784442424264D80000EA
:10221600000000000000003C427E0202423C00003A
:10222600000000F08808087E08080808083E00003C
:10223600000000000000007C22221C023C42423CBE
:10224600000000030202023A4642424242E7000010
:102256000000000C0C00000E08080808083E0000EC
:102266000000003030000038202020202020221ED0
:102276000000000302020272120A16122277000000
:102286000000000E0808080808080808083E0000B4
:10229600000000000000007F9292929292B7000028
:1022A600000000000000003B4642424242E70000B8
:1022B600000000000000003C42424242423C000056
:1022C600000000000000001B26424242221E0207B8
:1022D600000000000000007844424242447840E09A
:1022E60000000000000000774C040404041F0000F6
:1022F600000000000000007C42023C40423E00001C
:10230600000000000008083E080808080830000021
:1023160000000000000000634242424262DC00000E
:1023260000000000000000E7422424140808000012
:1023360000000000000000EB49495555222200002C
:10234600000000000000007624181818246E000013
:1023560000000000000000E74224241418080807C3
:10236600000000000000007E22100808447E0000E5
:1023760000C0202020202010202020202020C00067
:102386001010101010101010101010101010101047
:1023960000060808080808100808080808080600C3
:1023A6000C32C20000000000000000000000000027
:02AA89002000AB
:105BFA00240FFBE43AA3FAE0FEA3E0241F9002502C
:105C0A00FFE43EF0A3EFF022EEF0A3EFF0A3ECF0F6
:105C1A00A3EDF02290022AE0FEA3E0FFC390022740
:105C2A00E09FFF900226E09E90022CFEE0FCA3E09B
:105C3A00FD22900231E0FBA3E0FAA3E0F9022E284C
:105C4A00E0FCA3E0FD90022CE0FFA3E0900234CF39
:105C5A00F0A3EFF022900236E075F010A4FFE97C81
:105C6A00002FFFEC35F0FE74C62FF582741D3EF549
:105C7A0083E493900238F0E4A3F02275F008A4FFBD
:105C8A00900227E02FFF900226E090022835F0FECE
:105C9A00E0FCA3E0FD2290022CE0FEA3E0FF9002CC
:105CAA0027E02FFF900226E03E22FFE0FCA3E0FD62
:105CBA00D39FEE6480F8EC64809822E475F00102C8
:105CCA002EF79280C281D28122E4F0A3F0A3F0A33E
:105CDA00F022E0FAA3E0FBFFAE022290022CE0FEE3
:105CEA00A3E0FF22EF24E0FFE434FFFEEF78062270
:105CFA00E0FEA3E024C6F58274003EF583E493F93E
:105D0A00E4FA22FD7C0074017E00A8070822E0FE66
:105D1A00A3E0FFA3E0FCA3E0FD22FFE43EFE900225
:105D2A002FE02FF090022EE03EF022E0FAA3E0FFEF
:105D3A00AE0222C3E49FFFE49EF0A3EFF022A3EB9E
:105D4A00F0A3EAF0A3E9F022E0FCA3E0FDA3E0FE61
:105D5A00A3E0FF2212AA767F0302AA7612AA767F0E
:105D6A003102AA76A4FFE5F08FF0122EF7E422E0C2
:105D7A00FEA3E0FFD39400EE6480948022E0FFA3A8
:105D8A00E09002C7CFF0A3EFF022122F98E47B0A2B
:105D9A00FAF9F8022F98E0FF12AA76A3E0FF02AA06
:105DAA0076FFEE5CFEEF5D4E22A3EAF0A3EBF02253
:105DBA00ED9FFFEC9EF0A3EFF022FFEEF0A3EFF0D1
:015DCA0022B6
:04A688007F057E00CC
:10A68C00EF1FAC0670011E4C6010E4F5D875F9FC98
:0BA69C0075E966D2DE20DFE880FB22BB
:10A3DB008F20A207125CCCA206125CCCA205125CE9
:10A3EB00CCA204125CCCA203125CCCA202125CCCF9
:0BA3FB00A201125CCCA200125CCC227C
:04AA720012AA81FFA4
:05AA7600D28702A3DB02
:05A8BB00E0FEA3E0FF38
:10A8C000AD07AC06D287ECFF12A3DBAF0502A3DB1A
:05AA8100C28702A3DB07
:0AAA4D0012AA81AE04AF0502A8C0F2
:10A1980090024AEEF0A3EFF07F2A12AA8190024AB9
:10A1A800125DA0EAFF12AA76AF0312AA767F2B12DD
:10A1B800AA81ECFF12AA76AF0512AA769002501275
:07A1C8005DA07F2C02AA81BB
:10584600D2C620C65BE4FDFCFFFE12AA4D7BFF7AA2
:10585600AA7989E4FDFCFFFE12968490022A123092
:105866008100000000E490022EF0FDFCFFFE128C89
:1058760087E490022CF0FBFAFDFCFFFE129615E47D
:10588600FDFCFFFE129DB5E490022CF0A3F0FBFA9E
:10589600FDFCFFFE12989AE4FBFDFCFFFE1265D9A3
:1058A600D28612A688C28612A688D286D2C612A62A
:1058B60088C2C67FCB12AA817F3912AA767F2C12A4
:1058C600AA76E4FF12AA767F3412AA767F0212AA7B
:1058D600767FCF12AA727FC112AA767F3012AA767D
:1058E6007FE812AA817F8512AA76FF12AA767F78B0
:1058F60012AA767FEA12AA7212AA767FED12AA81FE
:105906007F64125D5E7F1212AA767F8112AA767F6D
:10591600F712AA817F2012AA767FC012AA817F235E
:1059260012AA767FC112AA817F1012AA767FC512AB
:10593600AA817F3E12AA767F2812AA767FC712AA6C
:10594600817F8612AA767F3612AA817F2812AA76CE
:105956007F3A12AA817F5512AA767FB112AA727F68
:105966001812AA767FB612AA817F0812AA767F82BB
:1059760012AA767F2712AA767FF212AA727F2612C1
:10598600AA817F0112AA767FE012AA817F0F125D9B
:10599600667F2B12AA767F0C12AA767F0E12AA7643
:1059A6007F0812AA767F4E12AA767FF112AA767F18
:1059B6003712AA767F0712AA767F10125D5E7F0ED7
:1059C60012AA767F0912AA76FF12AA767FE112AA98
:1059D600727F0E12AA767F14125D5E7F1112AA766E
:1059E6007F07125D667FC112AA767F4812AA767F6C
:1059F6000812AA767F0F12AA767F0C125D667F3692
:105A060012AA767F0F12AA767F1112AA817F78FEDC
:0D5A160012A68C7F2912AA817F2C02AA8182
:029E8700AC0627
:109E8900EC90022DF0A907900250E4F0A374EFF0D2
:109E99007B3F7A01E4FDFCFFFE12A198E4FBFA90F6
:109EA900022DE0FF12AA76AF0112AA760BBB0001C0
:109EB9000AEB64F04A70E80DBD00010CBC01DDBD80
:029EC90040DA7D
:019ECB002274
:108B5D00900226EEF0A3EFF090022AEBF09002289F
:058B6D00ECF0A3EDF0A7
:108B720090022D74FFF0A37418F0A374C6F0900253
:108B820026125D35C006C007241F125BFCD007D039
:108B92000612A19890022AE075F08090022E125DD2
:108BA2006E90022CF0E490022BF090022BE0FFC3B7
:108BB2009408502A90022D125C3F125D0D8005C36D
:108BC20033CE33CED8F9125DAB60059002C7800375
:108BD2009002C912A8BB90022BE004F080CC900254
:108BE2002E125CC590022CE004F0E0C3948040B5E4
:018BF2002260
:10A43000AB07AA068D828C83C006C007AE83AF82AD
:10A44000900250EEF0A3EFF0D007D00612A1989042
:0AA4500002C7E0FEA3E0FF02A8C06F
:109DB500AB07AA068D828C83EB24FFFFEA34FFFEF6
:109DC500C006C007E58224FFFDE58334FFFCEB24D4
:109DD50001FBE43AFAAE83AF82EF240190022C1224
:109DE5005C0A9002C7E0FFA3E090022ECFF0A3EF3C
:089DF500F0D007D0060293DE56
:0993DE00900226125C12125DB32C
:1093E700C007A3E0FFA3E0900250CFF0A3EFF0D0B7
:1093F7000712A198900228E0FFA3E0900230CFF077
:10940700A3EFF090022CE0FEA3E0FFD3900231E03F
:109417009F900230E09E5034900226E0FEA3E0FBCE
:10942700AA06C390022BE09B90022AE09A400D9077
:10943700022E12A8BB0BBB00010A80E6900231E0A6
:0C94470004F070BF900230E004F080B729
:0194530022F6
:06675C0090022E125C12F7
:10676200900238125CD390022EE0FEA3E0FFC3EB4E
:106772009FFFEA9E90023CF0A3EFF0900230E0FA15
:10678200A3E0FBC3900235E09BFE900234E09A90B6
:10679200023EF0A3CEF090022EE0FFA3E09002466C
:1067A200CFF0A3EFF0125DB390023C125D79400A84
:1067B200900242E4F0A304F0801AEF4E70089002B7
:1067C20042F0A3F0800E74FF900242F0A3F0900218
:1067D2003C125D3D90023E125D79400A900244E413
:1067E200F0A304F0801AEF4E7008900244F0A3F078
:1067F200800E74FF900244F0A3F090023E125D3DC1
:1068020090023EE0FEA3E090023C125CB490024093
:106812004007ECF0A3EDF08005EEF0A3EFF0E4907A
:106822000236F0A3F0900241E02401FF900240E022
:106832003400FED3900237E09F900236E09E400380
:106842000268DA900246125D1812A43090023CE00F
:10685200FEA3E0FF900239E02FF0900238E03EF014
:1068620090023EE0FEA3E0FF90023BE02FF0900298
:106872003AE03EF0900240E0FEA3E0900238125C63
:10688200B4401A900238125DBA900242E0FEA3E0D0
:10689200FF900247E02FF0900246E03EF090024067
:1068A200E0FEA3E0FF90023A125CB5401A90023A71
:1068B200125DBA900244E0FEA3E0FF900249E02F8D
:1068C200F0900248E03EF0900237E004F07006904B
:0868D2000236E004F002682721
:0168DA00229B
:10989A0090022AEAF0A3EBF0900226125C12C007AB
:1098AA00A3E0FAA3E0FB900228125C52D0071267E9
:1098BA005C900226125CDCC007A3125C4AD0071235
:1098CA00675C90022CE0FCA3E0FD90022AE0FAA378
:1098DA00E0FBA3125C52900226E0FEA3E0FF1267AF
:1098EA005C90022A125CDCC007900228125C4AD003
:0498FA000702675C9E
:0665D900900226125C1284
:1065DF00E4A3F0A3F0EBFF7E00A3EEF0A3EFF02512
:1065EF00E0FFEE33FEC374039F90022FF0E49E9002
:1065FF00022EF0125CE5D390022BE09FEE6480F840
:10660F0090022AE064809840030266DF12670C1242
:10661F005CA090022A125C3512674B125C1E90022E
:10662F0029E02DFD900228E03CFC12A430125CE51D
:10663F0012670C125C1E12674B125CA0126732902D
:10664F00022A125CA3125C32C3900229E09DFD90D6
:10665F000228E09CFC12A4301266E0125CE5C390A5
:10666F000227E09FFF900226E09E12673290022BD6
:10667F00E004F0700690022AE004F0C390022EE0CE
:10668F0064809480501790022AE0FEA3E07802C342
:10669F0033CE33CED8F92406125D24802D125CE55B
:1066AF00C390022BE09FFF90022AE09EFEEF78023C
:1066BF00C333CE33CED8F9240A125D2490022DE0D5
:1066CF0024FFF090022CE034FFF01266E002660225
:1066DF002290022AE0FEA3E0FF900227E02FFF9016
:1066EF000226E03EFE90022CE0FCA3E0FD90022982
:1066FF00E02DFD900228E03CFC12A43022C3900252
:10670F0027E09FFF900226E09EFE90022AE0FCA366
:10671F00E0FDC3900229E09DFD900228E09CFC1251
:10672F00A43022FE90022AE0FCA3E0FD900229E0B3
:10673F002DFD900228E03CFC12A43022C3900229C8
:0D674F00E09DFD900228E09CFC12A4302289
:09744900900232125C12A3EBF078
:10745200900232E0FEA3E090023A125DC49002C7AD
:10746200E0FDA3E090023CCDF0A3EDF0D3EF943821
:10747200EE94014003027569900234E0FCA3E0FD42
:1074820094E0EC94004003027569900236E024E037
:10749200F0900232125D35C006C0072407FBE43AC1
:1074A200FAA3E0FEA3E0240F125C07D007D0061275
:1074B200A198900237E07062F9125C5F900238E0A6
:1074C20030E00590023C80039002C9125D87900271
:1074D200C712A8BB900238E0C313F0900233E00455
:1074E200F07006900232E004F0900239E004F0E01D
:1074F200C3940840C790023AE0FFA3E0900232CF63
:10750200F0A3EFF0900235E004F07006900234E050
:1075120004F009E9641070A18047E4F9125C5F90FD
:107522000239E0FFC394085033900238E030E01F84
:10753200900233E02FFF900232E03400FEE9FD902A
:107542000235E02DFD900234E03400FC12A43090AC
:107552000238E0C313F0A3E004F080C309E9B410D9
:07756200BB90023C125D87A3
:0175690022FF
:089F0D00900232EFF0A3EDF029
:109F1500A312308100000001900233E0FF14F0EF3E
:109F25006020A3E0F8A3E0F9A3E0FAA3E0FB900228
:109F350032E0FFE4FCFDFE122F0D90023412307565
:089F450080D6900234125D5237
:019F4D0022F1
:068C8700900226125C12AF
:108C8D00E4900231F090022AA3125D57E4FCFD90AE
:108C9D00022A123075E490022FF090022EE0FFA30D
:108CAD00E0FEC39F5067C3EF9E14FD7F0A129F0D18
:108CBD00A804A905AA06AB0790022A125D52125DFF
:108CCD0094900230EBF0A3E0702490022EE014FF9C
:108CDD00A3E0FEC39F5017A3E0700DEE125C85E478
:108CED00900237F07B2080199002317401F09002D0
:108CFD002FE0125C85900230E02430FBE4900237C7
:0D8D0D00F012744990022FE004F0028CA7D0
:018D1A002236
:09961500900226125C12125DB3F2
:10961E00E490022DF090022CE0F9A3E0FFC39950E4
:10962E0054C3E99F14FD7F0A129F0DA804A905AA31
:10963E0006AB0790022AE0FEA3E0FFE4FCFD125DFC
:10964E0094AF0390022EEFF090022DE075F008A477
:10965E00FF900227E02FFF900226E0900228125C76
:10966E0097EB2430FBE4900237F012744990022DF0
:05967E00E004F080A0F3
:0196830022C4
:10968400900226125C12125D4890022A125C3FFB83
:10969400605AD3900227E09438900226E094014067
:1096A40012E4F0A3F0900229E02410F0900228E0E4
:1096B4003400F0D3900229E094E0900228E0940072
:1096C4004006900226125CD3900226125D18E490A4
:1096D4000237F0127449900227E02408F090022621
:0D96E400E03400F090022B125CC5809D2246
:1086430090029EEEF0A3EFF09002A2EBF09002A056
:05865300ECF0A3EDF0C6
:108658009002A574FFF0A37400F0A374C6F0900212
:108668009E125D35C006C007125BFAD007D006120D
:10867800A1989002A2E0C394205003743FF09002A6
:10868800A2E0D3947F4003743FF09002A2E0125C12
:10869800EFC333CE33CED8F9FF9002A6EE125D7247
:1086A8009002A4F0E49002A3F09002A3E0FFC39428
:1086B80008502A9002A5125C3F125D0D8005C33355
:1086C800CE33CED8F9125DAB60059002C780039017
:1086D80002C912A8BB9002A3E004F080CC9002A6C5
:0F86E800125CC59002A4E004F0E0C3944040B5DA
:0186F7002260
:108D1B0090022DEEF0A3EFF0900231EBF090022FCA
:058D2B00ECF0A3EDF0E7
:108D300090023474FFF0A37400F0A37446F0900224
:108D40002D125D35C006C007125BFAD007D006129F
:108D5000A198900231E075F040900235125D6E905E
:108D60000233F0E4900232F0900232E0FFC3940844
:108D7000502A900234125C3F125D0D8005C333CE41
:108D800033CED8F9125DAB60059002C78003900224
:108D9000C912A8BB900232E004F080CC90023512D8
:0E8DA0005CC5900233E004F0E0C3944040B59F
:018DAE0022A2
:0981740090022D125C12125D480C
:10817D00125C3C7003028258D390022EE094309032
:10818D00022DE094014012E4F0A3F0900230E024BF
:10819D0020F090022FE03400F0D3900230E094D024
:1081AD0090022FE094004007E490022D125CD490D1
:1081BD00022D125CDCC006C007125D1DEB240FFB07
:1081CD00E43A90022F125C00D007D00612A198124B
:1081DD005C3CFFC3942050027F3FEFD3947F40025D
:1081ED007F3F125CEEC333CE33CED8F990023412FA
:1081FD005DC4E4FB900234125CFA74017E00A802A7
:10820D00088005C333CE33CED8F9FFE9FDEF5D60AD
:10821D00059002C780039002C912A8BB0AEAB408F0
:10822D00D9900235E004F07006900234E004F00BB2
:10823D00EBB440C090022EE02410F090022DE034FB
:0B824D0000F0900232125CC502817D3F
:018258002203
:097AB800900221125C12125D48DB
:107AC100A3E07003027BBAE4900229F0900228E05F
:107AD100FFA3E0C39F4003027BBA900222E09430EF
:107AE100900221E094014012E4F0A3F0900224E01E
:107AF1002420F0900223E03400F0D3900224E0949B
:107B0100D0900223E094004007E4900221125CD45B
:107B1100900221125CDCC006C007125D1DEB240F30
:107B2100FBE43AFA900223125C01D007D00612A1BD
:107B310098900225125C3FFFC3942050027F3FEFD3
:107B4100D3947F40027F3F125CEEC333CE33CED855
:107B5100F9FF90022AEEF0A3EFF0E4FB90022A1263
:107B61005CFA74017E00A802088005C333CE33CECF
:107B7100D8F9FFE9FDEF5D60059002C7800390022F
:107B8100C912A8BB0AEAB408D990022BE004F0702C
:107B91000690022AE004F00BEBB440C0900222E010
:107BA1002410F0900221E03400F0900226125CC50E
:097BB100900229E004F0027ACDF3
:017BBA0022A8
:10906D004D73673A00416E74005758004469676943
:10907D0000436172005765617468657220537461B5
:10908D0074696F6E004E6F20636F6E6E65637469E9
:10909D006F6E212000576561746865720025005060
:1090AD006F77203A00706100446972203A00576969
:1090BD006E643A002F006D2F73005261696E3A0095
:1090CD006D6D00204720502053006B6D2F68004EB2
:1090DD00005300450057006D005354415455532023
:0490ED004F4B2100C4
:10382300900217E0FBA3E0FAA3E0F990021DE0F594
:1038330082758300122E41FF90021BE0241FF58244
:10384300E43402F583EFF090021BE004F090021DD4
:10385300E004F090021CE004F0E02290021BE0245C
:103863001FF582E43402F583E4F0900220E024D0D3
:10387300FFE434FFFE7C007D0A122E90AA06AB07FC
:1038830090021FE024D0FFE434FFFE7D64122E90EB
:10389300EF2BFFEE3AFE900221E024D0FDEC34FF43
:1038A300CD2FFFED3E900229F0A3EFF0900229E027
:1038B300FCA3E0FDE4122C297B4A7A0C7982783E42
:1038C300122A7E122C6290022BEEF0A3EFF09002EC
:1038D30025EEF0A3EFF0900225E0FAA3E0FB7C00D5
:1038E3007D64FFAE02122EA27C007D0A122EA2ED91
:1038F300243090021FF0AF037C007D0AAE02122E2B
:10390300A27C007D0A122EA2ED243022E02416F5BB
:1039130082E43402F583EEF090020DE004F0EF75DB
:10392300F00A8475F00A84E5F02430FEE02416F5ED
:1039330082E43402F583EEF090020DE004F0EF75BB
:10394300F00A84E5F02430FEE02416F582E4340224
:10395300F583EEF090020DE004F02290021BE024C8
:103963001FF582E43402F583E4F0900220E024D0D2
:10397300FFE434FFFE7C007D0A122E90AA06AB07FB
:1039830090021FE024D0FFE434FFFE7D64122E90EA
:10399300EF2BFFEE3AFE900221E024D0FDEC34FF42
:1039A300CD2FFFED3EFE900225F0A3EFF0227474BD
:1039B3002FF582E43402F583E0FF900210E0241136
:1039C300F582E43402F583EFF0900210E0042274F0
:1039D300002DF582E43400F583E0FF900210E0242B
:1039E30015F582E43402F58322122A7E122C6290AA
:1039F300021DEEF0A3EFF0900221E0FCA3E0FD90A6
:103A0300021BE0FEA3E0FF90021FE0FAA3E02FFBFE
:103A1300EA3EFA90021DE0FEA3E0FF900221E0F8E7
:103A2300A3E0C39FFFE89E900234F0A3EFF090025F
:103A33001FE0FEA3E0FF22E49002C9F0A3F074FFAD
:103A43009002C7F0A3F022FDAC06E4122C297B7B85
:103A53007A1479CE783F122A7E7466FBFAF978409D
:103A6300122B87122C62900227EEF0A3EFF0229024
:103A73000210E02411F582E43402F583E4F07B01C3
:103A83007A02791122900223E0FCA3E0FDE4022CE8
:103A93002990021BE0241FF582E43402F583E4F04D
:103AA30090021FE02290021DF0E490021CF022EF2E
:103AB300F0900210E004F02274FF9002C7F0A374A8
:103AC300E0227B017A0279BA7C007E002290021FF9
:103AD3007420F0900227E0FEA3E0FF22FFE433FE10
:103AE30090020FE0FDC39FEE6480F87480982290EB
:103AF30002277D0AE0FAA3E0FB7C00FF2290021F6D
:103B0300F07C007D0AAF03AE0222F090020FE004C6
:103B1300F022F09002C774F8F0A3E4F022A3F0902F
:103B23000225E0FEA3E0FF22F07B017A0279152251
:103B3300122A7E122C6290021BEEF0A3EFF0227B7E
:103B4300FF7D807C00E4FFFE22E4900210F09002EF
:103B53000F22F0E02411F582E43402F583E4227CA1
:103B6300007F327E00227BFF7C007F107E0122904B
:103B73000221F0E4A3F090021FE022F090020FE094
:103B830004F022C3940AEE9400229002C7E4F0A347
:0B3B9300741FF02290020FE0FFC3221D
:105231007F337E0012A88EEF640260030254469011
:1052410002A8E0640560197405F0E4FFFE129E8770
:105251007407123ABDF07A90796D123B4212817453
:10526100E490020FF090020FE0FFC3940C500C7415
:10527100152F1239E4E4123B0D80EAE4900210F09C
:1052810090020F7407F090020FE0FFC3940D5020BD
:1052910074002FF582E43400F583E0C3139002110A
:1052A100F0642060061239DC123AB2123B0E80D64D
:1052B10090000DE0541EC313900211F0D3940040EE
:1052C1003C1239DE742D123AB3A3E0FFC3940A50A5
:1052D10009EF2430FF900210801D900211E0FF754C
:1052E100F00A842430FE1239DEEE123AB3EF75F083
:1052F1000A84E5F02430FF1239E1123AB21239DEA4
:10530100E4F0123A3B123B2CE4FDFCFFFE128174E7
:10531100900212740DF0E4A3F0900213E0C394061E
:105321004003025446900212E0FF2400F582E43467
:1053310000F583E020E00302543AE4900210F012F9
:1053410039E17420123AB3EF240490020FF0900275
:1053510012E0240C123ADF500B1239D2123AB21277
:105361003B0E80EA1239DEE4F09002C7F0A3741F0D
:10537100123B2B7D207C007FA07E00128174E49083
:105381000210F0900212E0240D90020FF090021230
:10539100E02416123ADF500B1239D2123AB2123B04
:1053A1000E80EA1239DEE4123B2B7D40FC7FA0FE29
:1053B100128174123A41900212E02416F582E4340B
:1053C10000F583E0900214F024DD601C24E56020E8
:1053D10024DF600C24ED70217BFF7A9079728016B6
:1053E1007BFF7A907976800E7BFF7A9079798006BF
:1053F1007BFF7A90797EE4800B900214E0A3F0E4C5
:10540100A3123B2BFDFC7FFAFE128174900212E085
:105411002417F0E0FD900100E0C39D900210F074AC
:10542100002DF9E43400FA7B01E0900228F07D8040
:105431007C007F507E00027AB8900212E0240712AD
:055441003B0D02531AAF
:015446002243
:0E3B9E00900217EBF0A3EAF0A3E9F0A3EDF01C
:103BAC007F337E0012A88EEF64026003023E957F85
:103BBC000B7E0112A88EEF7003023E9590021AE064
:103BCC0070309002A8E0640260097402F0E4FFFE19
:103BDC00129E87123A3AFB7A9079827D32123B62BE
:103BEC001281747BFF7A9079927D647C007F320223
:103BFC003E909002A8E064037003023CA77403F0AB
:103C0C00E4FFFE129E87E49002C9F0A3123B157BE1
:103C1C00FF7A9079A2FDFCFFFE128174123A41E406
:103C2C00FBFDFC7F307E01128D1B7A9079AA7D20E2
:103C3C007F30123ED67A9079AC7D40123EE07A907D
:103C4C0079B27D407F20123ED67A9079B57D601294
:103C5C003EE07B017D607C007FA07E00128D1B7A94
:103C6C009079BB123B421281747D80123EC67A90D1
:103C7C0079C37D80123B691281747BFF7A9079C77E
:103C8C007DA07C00E4FFFE1281747DA0123EC67AFA
:103C9C009079CD7DA0123B69128174123ABBF0E48D
:103CAC0090021BF0740D123AA8123823B403FA12C6
:103CBC00395EC39420EE94005015123B22C374203D
:103CCC009FF0E49E900225F0E490021EF080149088
:103CDC000226E024E0F0900225E034FFF090021E72
:103CEC007401F0900225123A8B7B667A6679E6783D
:103CFC003F123A6390021EE07006A3742DF080060A
:103D0C0090021F7420F0123AD6123B86500C90028F
:103D1C00207420F07C007D0A8012900227E0FAA328
:103D2C00E0FBFF1238FB900220123B03123908A370
:103D3C00F0E4A3F07B017A02791FE4FDFC7FE0FE46
:103D4C00128174E490021BF07419123AA8123823F1
:103D5C00B402FA123A94B430037420F07D207FF050
:103D6C00123EEBE490021BF090021D741C123AAB55
:103D7C00123823B404FA123A94B430037420F07D50
:103D8C00407FD0123EEB128BF37D407F60123AC520
:103D9C00128174E490021BF090021D04123AAB12D3
:103DAC003823B403FA123A94B4300B7420F0A3E025
:103DBC00B430037420F07D60123E967405123AAB59
:103DCC00123823B403FA12395E123A4A123B865067
:103DDC000B123AD0123904900220800D123AF212D2
:103DEC0038FF123B00123908A3F0E4A3F07F7012E5
:103DFC003EAE7409123AAB123823B403FA12395E90
:103E0C00123A4A123B86500B123AD01239049002E5
:103E1C0020800D123AF21238FF123B00123908A31F
:103E2C00F0E4A3F07FD0123EAE7411123AAB12380C
:103E3C0023B403FA12385E123B20123904123B727F
:103E4C00B4300B7420F0A3E0B430037420F07DA0E8
:103E5C00123E967415123AAB123823B403FA123888
:103E6C005E123B20123904123B72B4300B7420F0FA
:103E7C00A3E0B430037420F07B017A02791F7DA09B
:093E8C007C007FC07E00128174ED
:103E9500227B017A02791F7C007F607E001281748B
:103EA500E490021BF090021D227B017A02791F7DAE
:103EB500807C007E00128174E490021BF090021D4C
:103EC500227BFF7A9079C17C007FA07E00128174ED
:103ED500227BFF7C007E01128174227BFF7C00E443
:103EE500FFFE128174227B017A02791F7C007E001D
:043EF50012817422A0
:104DE9007F337E0012A88EEF64026003024FE97FD1
:104DF9008D7E0112A88EEF7003024FE99002A8E0A0
:104E0900640460597404F0E4FFFE129E87123A3A72
:104E1900FB7A9079D0E4FDFCFFFE128174123ABB53
:104E2900F07B321250017B33125001123A41E49067
:104E39000237F07B4E7D74124FF47B537DD8124FAD
:104E4900F47B577DA6FC7FC8FE127449E4900237B3
:104E5900F07B457DA6FC7F2C7E01127449128BF3F1
:104E6900123A417B017A0279BAE4FDFC7F187E018E
:104E7900129684E4900210F09002527D64123AF77F
:104E8900AE02122EA2EF24301239BC1238F8FF12EA
:104E990039C0F0900252E0FEA3E0FF123904123942
:104EA900BC123B55123A40123A817DBE7C007FF21A
:104EB9007E00129684900252E0FFA3E09002A9CFEF
:104EC900F0A3EFF01279B390025BE0FF7E00FD7C66
:104ED90000E4122C297B667A6679E6783F122A7EED
:104EE900122C62AB07AA06E4900210F0FC7D641252
:104EF9003901FF1239C01238F8FF1239C0F0AE0279
:104F0900AF03123904FF1239C0123B55F090021158
:104F1900E0B4300B7420F0A3E0B430037420F01235
:104F29003ABB123A807F0A124FEA7BFF7A9079D70F
:104F39007F4A124FEA123B8D90027BE07BFFB44E11
:104F4900067A9079DC80047A9079DE7DA012500D82
:104F5900123B4CF0123B97940750081239B1123B9F
:104F69007E80F1123A727DA0FC7F40FE128174901E
:104F79000285E07BFFB445067A9079E080047A9057
:104F890079E27DC812500D123B4C7409F0123B971F
:104F9900941150081239B1123B7E80F1123A727D98
:104FA900C8FC7F30FE128174123B4CF0123B97947F
:104FB90006501074542FF582E434021239B9123BA9
:104FC9007E80E9123A727D20FC7FB0FE1281747BEB
:104FD900FF7A9079E47D207C007F307E0112817414
:104FE900227D507C007E0012817422FC7FFEFE121D
:104FF9007449E4900237F0227DAE7C007FFE7E008A
:0E5009001265D9227C007F0A7E00128174227B
:106D0A007F337E0012A88EEF64026003026E5A90EF
:106D1A0002A87401F0125846E4FFFE129E87123A46
:106D2A003AE4900210F0A3F0A3F0A3F090020FF05F
:106D3A0090020DF0900210E0FEA3E0FFA3E0FCA396
:106D4A00E0FD90020FE0FB128B5D900211E024201F
:106D5A00F0900210E03400F090020FE0041239566D
:106D6A00E0C3940A40CE123ABBF07BFF7AA5798938
:106D7A007D327C007F147E00128174E490020EF052
:106D8A0090020EE0FFC39410501474162FF582E49B
:106D9A003402F583E4F090020EE004F080E29002FF
:106DAA0014E4F0A37410F0FF7E0012A88EE490029F
:106DBA000DF0EF75F064842430FE12390F9002153D
:106DCA00E004F07006900214E004F0E490020EF081
:106DDA0090020DE02416F582E43402F583742E1233
:106DEA003956900214E0FEA3E0FF12A88EEF75F068
:106DFA0064842430FE90020D12390F900215E004CB
:106E0A00F07006900214E004F090020EE004F0E044
:106E1A00C3940340BB128BF37D327FDC123AC51256
:106E2A008174123B167B017A0279167D64FC7F1EFF
:106E3A00FE128174123B8D7BFF7A9079E67DC8122F
:106E4A003B62128174E49002A9F0A3F0A3F0A3F0CC
:016E5A002215
:1079B30090021FE4F0A374FEF0A3E4F0A374AEF00E
:1079C300A3E4F0A37428F09002ABE0FCA3E0FD90E5
:1079D30002A9E06C7003A3E06D7003027A71E412F4
:1079E3003A43127A9CC004C005C006C007123A8805
:1079F300D003D002D001D000123B339002AB127AF5
:107A030072C004C005C006C007123A88D003D00272
:107A1300D001D0001239EC12675C9002A9E0FCA3FC
:107A2300E0FDA3ECF0A3ED123B15127A9CC004C059
:107A330005C006C007123A88D003D002D001D00097
:107A4300123B339002A9127A72C004C005C006C06B
:107A530007123A88D003D002D001D0001239EC12B9
:0E7A6300675C123A31A3E0FCA3E0FD129DB572
:107A710022E0FEA3E0FFC3745A9FFDE49EFCE412E2
:107A81002C297BC37AF579487840122A7EE4FBFAE7
:107A910079347843122B8712632C22122C297BC351
:107AA1007AF579487840122A7EE4FBFA79347843F2
:077AB100122B8712632C2247
:1030B2004750532000B1B1CEB33A2000C4CFCEB3B3
:1030C2003A2000B6ABBEAD3A2000CEF7BEAD3A20F4
:1030D20000BAA3B0CE3A2000202020415052532DF6
:1030E2003531544E4320202000535441545553202F
:1030F2004F4B21002020C6F8CFF3BDD3BFDAB0E595
:1031020020200020202020C3BBC1ACBDD3A3A1201E
:103112002000576561746865722053746174696F29
:103122006E004E6F20636F6E6E656374696F6E2101
:1031320020005765617468657200504D32353A203F
:103142003030300025007061004449523A00575334
:10315200203A002F00204D2F5300524E203A006D8E
:103162006D00504F533A00202020004D53473A0043
:10317200416E7400575800446967690043617200E8
:1031820000001800240024F4190C020404000400B6
:10319200040004000204010800F000000000000026
:1031A200000000000000000020202020200020005D
:1031B20050500000000000005050F850F8505000ED
:1031C2001038507028287000006868102058580085
:1031D2003028307048483000101000000000000015
:1031E200102020202020100020101010101020008D
:1031F200002070707020000000202070202000004D
:103202000000000000101000000000780000000024
:1032120000000000000020000808101020204000DC
:103222003048484848483000206020202020700064
:1032320030480810204078003048083008483000F4
:1032420010303050507810007840407008087000FC
:10325200304840704848300078480810202020004C
:103262003048483048483000304848380848300034
:10327200000020000020000000002000002040008C
:10328200081020402010080000007800780000009C
:103292004020100810204000304808102000200074
:1032A200304848582828380030484848784848006C
:1032B20070484870484870003048404040483000EC
:1032C2007048484848487000784040704040780054
:1032D20078404070404040003048405848483000F4
:1032E2004848487848484800702020202020700034
:1032F20008080808484830004848506050484800CC
:10330200404040404040780048787848484848006B
:1033120048686858584848007848484848487800FB
:10332200704848704040400030484848685838006B
:1033320070484870605048003048403008483000BB
:103342007820202020202000484848484848300063
:103352004848484830303000484848487878480063
:1033620048483030304848008888502020202000CB
:1033720078081030204078003020202020203000B3
:1033820080804040202010003010101010103000BB
:103392002050000000000000000000000000780043
:1033A20020200000000000000000003838483800EB
:1033B20040404070484870000000003840403800EB
:1033C20008080838484838000000003078403000CB
:1033D20000102078202020000000003848380830F3
:1033E200404040705050500000002000202020003B
:1033F200000010001010106040404058605048001B
:10340200202020202020700000000078585858000A
:103412000000007048484800000000304848300072
:1034220000000070484870400000003848483808E2
:103432000000005860404000000000386018700032
:10344200000020702020300000000048484838006A
:103452000000004848303000000000A8A87050006A
:10346200000000483030480000000048483808306A
:10347200000000781020780030202040202030000A
:10348200202020202020200060202010202060000A
:103492002850000000000000007070707070000082
:1034A200900217E0FBA3E0FAA3E0F990021DE0F519
:1034B20082758300122E41FF90021BE0241FF582C9
:1034C200E43402F583EFF090021BE004F090021D59
:1034D200E004F090021CE004F0E02290021BE024E1
:1034E2001FF582E43402F583E4F0900220E024D058
:1034F200FFE434FFFE7C007D0A122E90AA06AB0781
:1035020090021FE024D0FFE434FFFE7D64122E906F
:10351200EF2BFFEE3AFE900221E024D0FDEC34FFC7
:10352200CD2FFFED3EFEE4FD900229123075E47FBF
:10353200FEFEFDFC900229E0F8A3E0F9A3E0FAA365
:10354200E0FB122F0DE47BE87A03F9F8122F989032
:10355200022D12307590022DA3A3E0FFA3E090028A
:1035620025CFF0A3EFF0900225E0FAA3E0FB7C0068
:103572007D64FFAE02122EA27C007D0A122EA2ED05
:10358200243090021FF0AF037C007D0AAE02122E9F
:10359200A27C007D0A122EA2ED243022E02411F535
:1035A20082E43402F583EEF090020DE004F0EF7550
:1035B200F00A8475F00A84E5F02430FEE02411F567
:1035C20082E43402F583EEF090020DE004F0EF7530
:1035D200F00A84E5F02430FEE02411F582E434029E
:1035E200F583EEF090020DE004F02290021BE0243D
:1035F2001FF582E43402F583E4F0900220E024D047
:10360200FFE434FFFE7C007D0A122E90AA06AB076F
:1036120090021FE024D0FFE434FFFE7D64122E905E
:10362200EF2BFFEE3AFE900221E024D0FDEC34FFB6
:10363200CD2FFFED3EFE900225F0A3EFF022E02415
:1036420011F582E43402F583EFF0900210E004F009
:10365200E02411F582E43402F58322900233E0FB88
:10366200A3E0FAA3E0F9022E2874002DF582E434D7
:1036720000F583E0FF900210E02416F582E43402A4
:10368200F5832290022BFFF0900225E475F00102EF
:103692002EF7900239E0FEA3E024A2F58274313EB7
:1036A200F583E49322EFF0A3EDF0A3EBF0A3EAF0AD
:1036B200A3E9F02224E0FFE434FFFEEF780322FDC9
:1036C200900232E02433F582E43402F58322900240
:1036D2001DF0E490021CF022900237E004F0E004B6
:1036E200F0900236E004F022900228E004F0E004B8
:1036F200F0900227E004F022EFF0900210E004F0D4
:1037020022EFF0900210E0042290021BE0241FF549
:1037120082E43402F583E4F022900232E004F0E025
:1037220004F0900231E004F0227DA1122E900C7D73
:1037320068122EA2A3EEF0A3EFF022FF900237E070
:10374200243BF582E43402F583EFF090023AE00480
:10375200F022FF900228E0242DF582E43402F58362
:10376200EFF090022CE004F022A3F0900225E0FE9C
:10377200A3E0FF2274742FF582E43402F583E0FFA4
:1037820090021022900220F07C007D0AAF03AE026C
:10379200229002277D0AE0FAA3E0FB7C00FF22FFD1
:1037A200E433FE90020FE0FDC39FEE6480F8748064
:1037B20098227420F0900227E0FEA3E0FF22F0900E
:1037C200020FE004F022900239FFEEF0A3EFF022A4
:1037D200E4900237F0900236F022E4900228F09052
:1037E2000227F022E4900210F090020F22F07B01F7
:1037F2007A02791622EF25E0FF0EEE22F090020FF8
:10380200E004F022900221F0E4A3F090021FE022F3
:1038120090020FE0FFC322E4900232F0900231F0F6
:013822002283
:105DCB007F337E0012A88EEF64016003025F787F41
:105DDB008D7E0112A88EEF7003025F787F301292D6
:105DEB00EA7F011292EA7F0A7E0012A7AC7F0612AD
:105DFB0092EA7F0C1292EA129D6A7BFF7A3079B29B
:105E0B00E4FD7F011298FEE4900210F09002527DA7
:105E1B0064123798AE02122EA2EF2430FF900210BC
:105E2B00123652123703123587FF123652123703CE
:105E3B00F0900252E0FEA3E0FF123593FF900210A8
:105E4B00123640742012364BE4F07D03125F7990CA
:105E5B00025BE0FF7E007C007DB9122E907D641208
:105E6B002EA2AB07AA06E4900210F0FC7D6412355B
:105E7B0090FF123652123703123587FF1236521229
:105E8B003703F0AE02AF03123593FF123640744B5B
:105E9B0012364B746D12364BE4F07D05125F797B35
:105EAB000E7D08E4FF129A8190027BE07BFFB44EDB
:105EBB00067A3079B780047A3079BEE4FD7F02121E
:105ECB0098FE1237E6F01238129407500E123776FE
:105EDB001236521237031237FE80EB900210123635
:105EEB0052E4F07F02125F85900285E07BFFB445A0
:105EFB00067A3079C580047A3079CCE4FD7F0312C1
:105F0B0098FE1237E67409F01238129411500E12E3
:105F1B0037761236521237031237FE80EB9002108F
:105F2B00123652E4F07F03125F857BFF7A3079D310
:105F3B00E4FD7F041298FE1237E6F0123812940635
:105F4B00501674542FF582E4340212377E123652F7
:105F5B001237031237FE80E3900210123652E4F030
:0D5F6B007B017A0279117D037F041298FEFC
:105F7800227B017A0279117F011298FE227B017A35
:095F88000279117D031298FE223A
:107EA6007F337E0012A88EEF64016003027F9C126E
:107EB600A4AC7F011292EA7F0A7E0012A7AC7BFF78
:107EC6007A3079DA7F01129BE47BFF7AA579897F84
:107ED60002129BE4E490020EF090020EE0FFC394BF
:107EE60010501474112FF582E43402F583E4F090F7
:107EF600020EE004F080E290020FE4F0A37410F0AA
:107F0600FF7E0012A88EE490020DF0EF75F06484F7
:107F16002430FE12359E900210E004F070069002A6
:107F26000FE004F0E490020EF090020DE02411F54B
:107F360082E43402F583742E1235E590020FE0FEDA
:107F4600A3E0FF12A88EEF75F064842430FE900241
:107F56000D12359E900210E004F0700690020FE0BC
:107F660004F090020EE004F0E0C3940340BB128BD1
:107F7600F37B017A0279BA7D067F021298FE7B01B5
:107F86007A0279117F04129BE47BFF7A3079EB7DCC
:067F9600017F031298FEBA
:017F9C0022C2
:093EF9009002171236ADA3EDF0A2
:103F02007F337E0012A88EEF640160030241DF7FDF
:103F12000B7E0112A88EEF70030241DF7F301292F6
:103F2200EA7F011292EA7F0A7E0012A7AC7F061294
:103F320092EA7F0C1292EA129D6A90021AE0702BAA
:103F42007BFF7A3079F6FD7F011298FE7BFF7A3192
:103F520079057F0212422C7A3179147F0312422CA6
:103F62007A317924E4FD7F040298FE7A3179347F34
:103F7200011241F4740D1236D31234A2B403FA12B0
:103F820035EDC39420EE9400501512376DC37420A2
:103F92009FF0E49E900225F0E490021EF0801490BF
:103FA2000226E024E0F0900225E034FFF090021EA9
:103FB2007401F012376D7C007D0A122E907D121270
:103FC200373390021EE07006A3742DF08006900233
:103FD2001F7420F01237B7C3940AEE9400500C906D
:103FE20002207420F07C007D0A800F900227E0FA04
:103FF200A3E0FBFF12358A123786123597A3F0E44D
:10400200A3F07F011242167A317982E4FD7F071212
:104012009ADF7B0E7D08E4FF129A817A31793C7F28
:10402200021241F474191236D31234A2B402FA12F3
:10403200370B7B017A02791F7D067F021298FE7B85
:10404200FF7A3179467D077F021298FEE490021BC7
:10405200F0741C1236D01234A2B404FA12370B9048
:10406200021FE0B430037420F07F031242167A314B
:1040720079487D077F031298FE128BF37B017A0247
:1040820079BAE4FD7F09124234041236D01234A206
:10409200B403FA12370B90021FE0B4300B7420F015
:1040A200A3E0B430037420F07A31794B7D081242D8
:1040B200247D081241E074051236D31234A2B403EF
:1040C200FA1235ED12372B90021F7420F0C3EF94D1
:1040D2000AEE9400500CA31237B4123593900221C9
:1040E200800D12379312358E123786123597A3F050
:1040F200E4A3F07A3179507D101242247D101241EE
:10410200E074091236D31234A2B403FA1235ED1256
:10411200372BC3940AEE9400500E90021F1237B44C
:10412200123593900220801012379312358E90022E
:104132001F123789123597A3F0E4A3F07D101242C3
:10414200047D107F0D12756A7BFF7A3179577D10DD
:104152007F0E12423490021D74111236D31234A211
:10416200B403FA1234DD12376B123593123806B4E7
:10417200300B7420F0A3E0B430037420F07BFF7A9C
:1041820031795C7D187F0812756A7B017A02791F8A
:104192007D187F0A12756AE490021BF090021D746A
:1041A200151236D31234A2B403FA1234DD12376B6D
:1041B200123593123806B4300B7420F0A3E0B430F9
:1041C200037420F07D181242047D187F0D12756A67
:0D41D2007BFF7A3179617D187F0F12756ACD
:1041DF00227B017A02791F7F0A12756AE490021B13
:1041EF00F090021D227BFFE4FD1298FEE490021B6B
:1041FF00F090021D227BFF7A3179557F0C12756A80
:10420F007B017A02791F227B017A02791F7D0512C9
:10421F0098FE7BFF227BFF7F0812756A22E4FD1256
:0E422F0098FE7BFF2212756AE490021BF022BB
:1044F2007F337E0012A88EEF6401600302473E7F85
:104502008B7E0112A88EEF700302473E7F3012921B
:10451200EA7F011292EA7F0A7E0012A7AC7F06129E
:1045220092EA7F0C1292EA129D6A9002157408F0C8
:104532002408FD7BFF7A317964E4FF12756A9002E8
:1045420015E02410FD7BFF7A317969E4FF12756A68
:10455200E4FB7D107F08129A817BFF7A31796D7DB1
:10456200027F08126BA9E490020FF090020FE0FFA5
:10457200C3940C500C74162F12367DE41237C0808F
:10458200EAE4900210F090020F7407F090020FE03C
:10459200FFC3940D502074002FF582E43400F5839C
:1045A200E0C313900211F0642060061236751236D1
:1045B200FA1237C180D690000DE0541EC313900248
:1045C20011F0D39400403C123677742D1236FBA3BF
:1045D200E0FFC3940A5009EF2430FF900210801DBF
:1045E200900211E0FF75F00A842430FE123677EE55
:1045F2001236FBEF75F00A84E5F02430FF12367AAA
:104602001236FA123677E41237EF7F01129BE490EA
:104612000212740DF0E4A3F0900213E0C39406407A
:104622000302473E900212E0FF2400F582E43400C8
:10463200F583E020E003024732E4900210F01236E4
:104642007A74201236FBEF240490020FF0900212CB
:10465200E0240C1237A1500B12366B1236FA1237C5
:10466200C180EA123677E4F0900215E02408FD12C8
:1046720037F07F0312756AE4900210F0900212E0A4
:10468200240D90020FF0900212E024161237A1506E
:104692000B12366B1236FA1237C180EA123677E401
:1046A200F0900215E02410FD1237F07F0312756AB4
:1046B200900212E02416F582E43400F583E09002C1
:1046C20014F024DD601C24E5602024DF600C24ED5E
:1046D20070207BFF7A31797280257BFF7A3179767F
:1046E200801D7BFF7A31797980157BFF7A31797E63
:1046F200800D900214E0900216F0E4A31237EF7DD1
:10470200067F011298FE900212E02417F0E0FF905B
:104712000100E0C39FFE900210F074002FF9E43410
:1047220000FA7B01900227EEF07D027F0A02825995
:0C473200900212E024071237C002461A61
:01473E002258
:079BE400900222EF1236ABE4
:109BEB007F301292EA900222E024FE600E14600F86
:109BFB00146010240370117F80800A7F9080067F91
:109C0B008880027F981292EAE4900226F090022359
:109C1B00123660FF601612936490022412368D90F8
:0C9C2B000226E004F0E0D3941040E22296
:019C3700220A
:0698FE009002311236A7B2
:109904007F301292EA900231E024FE601214601754
:1099140014601C24037022900232E024808016908C
:109924000232E02490800E900232E0248880069077
:109934000232E02498FF1292EAE4900236F0900298
:1099440033123660FF601612936490023412368D1F
:0D995400900236E004F0E0D3941040E222CF
:0199610022E3
:069ADF009002311236A7CF
:109AE500E4A3F07F341292EA900232E02480FF1260
:109AF50092EA900231E02480FF1292EA7F301292BE
:109B0500EA900233123660FF1293649002341236E3
:109B15008D900233123660FF129364900234123630
:109B25008D900232E004F0900236E004F0E0C39438
:039B35001040B02D
:019B3800220A
:0A9A8100900232EBF0900231EFF09A
:109A8B00C3ED9F900234F0E4900233F0900234E087
:109A9B00FF900233E0C39F50367F341292EA90025C
:109AAB0032E02480FF1292EA900231E02480FF1210
:109ABB0092EA7F301292EA7FFF1293647FFF129338
:109ACB0064900231E004F0900233E004F080BD7F3B
:049ADB00360292EAD3
:06756A009002311236A769
:1075700012365D7003027634900232E0900238F0E9
:10758000E4900236F0900236E0FFC394105010747D
:107590003B2FF582E43402F583E41236E280E612F2
:1075A000365D1236B6C333CE33CED8F91237C81291
:1075B00037D212369412373D7006900239E004F04B
:1075C0001236DAE0B408EB90023412368D12365DD2
:1075D00070131237D3127639A31236E0E0C3940841
:1075E00040F302763412365D1236B6C333CE33CE54
:1075F000D8F91237C89002377401F0E4900236F0DF
:1076000012369412373D7006900239E004F01236BB
:10761000DAE0B408EB1237D2127639A31236E0E082
:10762000C3940840F390023412368D900231E00486
:09763000F00275707F360292EA47
:107639007F341292EA900238E02480FF1292EA9095
:107649000231E02480FF1292EA7F301292EA90021E
:1076590037E0243BF582E43402F583E0FF129364BA
:10766900900237E004F0E0243BF582E43402F5832C
:0C767900E0FF129364900237E004F0225E
:068259009002221236A77C
:10825F00A3E0700302832D900227E0FFC313900267
:10826F0029F0EF5401A3F0E4900228F0900229E0E6
:10827F00FF900228E0C39F506E90022412366012C6
:10828F003685EF640D700302832D90022BE0FE64A0
:10829F000A700302832D90022412366090022C1272
:1082AF003688BF0D0690022C7420F090022CE0B49B
:1082BF000A037420F0900222E0FFA3E0FDAB0690CA
:1082CF00022CE0900230F01284BE900222E004F003
:1082DF00E0D3940F40087408F0A3E02408F0900254
:1082EF0028E004F002827B90022AE0602C900224A6
:1082FF00123660123685EF640D602390022BE0FB7F
:10830F00640A601AE490022CF0900222E0FFA3E0CE
:0E831F00FDE4900230F01284BE7F361292EA26
:01832D00222D
:0884BE0090022DEFF0A3EDF098
:1084C600E4900231F0900231E0FFC39410500C7436
:1084D600332F1236C8E412372380EAEB1236B6C3BE
:1084E60033CE33CED8F9FF12381974A22F12369D27
:1084F6001236C1EDF00FBF00010E12371BE0B408B3
:10850600E9900230E0FD602D1236B6C333CE33CE8D
:10851600D8F9FF9002327401F0E4900231F074A2AF
:108526002F12369D1236C1EDF00FBF00010E123725
:108536001BE0B408E91238197F341292EA90022E31
:10854600E02480FF1292EA90022DE02480FF12922E
:10855600EA7F301292EA1236C21285751236C512B9
:0E856600857590022E123721E0C3940840CA9A
:0D85740022E0FF129364900232E004F02236
:0E6BA9009002241236AD900222EFF0A3EDF020
:106BB700900229EFF0A3EDF09002241236607003E3
:106BC700026CB9E4900227F0900227E0FFC394100B
:106BD7005010742D2FF582E43402F583E41236F257
:106BE70080E69002241236601236B6C333CE33CE17
:106BF700D8F990022B1237CB1237DC90022B1236C2
:106C070097123754700690022BE004F01236EAE030
:106C1700B408E890022512368D900224123660706F
:106C2700151237DD126CBE90022A1236F0E0C394BB
:106C37000840F1026CB99002241236601236B6C3CE
:106C470033CE33CED8F9FF90022BEEF0A3EFF090BE
:106C570002287401F0E4900227F090022B12369775
:106C6700123754700690022BE004F01236EAE0B4B3
:106C770008E81237DC126CBE90022A1236F0E0C325
:106C8700940840F1900222E004F090022512368D1C
:106C9700900222E0D3940F400E7408F090022AE08D
:106CA700900223F0026BBF900223E090022AF002C9
:076CB7006BBF7F360292EA79
:106CBE007F341292EA90022AE02480FF1292EA9028
:106CCE000222E02480FF1292EA7F301292EA9002B2
:106CDE0028E0242DF582E43402F583E0FF1293645C
:106CEE00900228E004F0E0242DF582E43402F583CE
:0C6CFE00E0FF129364900228E004F022F2
:10A4AC007F301292EA7F0112A4CA7F0612A4CA7FDF
:10A4BC000C1292EA7F0A7E0012A7AC029D6A1292DD
:09A4CC00EA7F0A7E0012A7AC220F
:109D6A00E4900232F0E4900231F07F341292EA90E9
:109D7A000232E02480FF1292EA900231E02480FF4E
:109D8A001292EA7F301292EAE4FF129364E4FF121D
:109D9A009364900231E004F0E0C3941040CC900246
:0A9DAA0032E004F0E0C3942040BB57
:019DB400228C
:1092EA00D280E4FEC28100D281000EEEB405F5C23E
:1092FA0080C280C28100D28100C280C28100D28134
:10930A0000C280C28100D28100E4FEEF30E704D2BD
:10931A00808002C280C28100D281001237F7B40471
:10932A00EAC280E4FEC28100D281000EEEB404F5E6
:10933A00E4FEEF30E704D2808002C280C28100D20C
:10934A0081001237F7B404EAC280E4FEC28100D277
:0A935A0081000EEEB404F502A92F05
:10936400D280E4FEC28100D281000EEEB405F5C2C3
:1093740080C280C28100D28100D280C28100D281A9
:1093840000C280C28100D28100E4FEEF30E704D243
:10939400808002C280C28100D281001237F7B404F7
:1093A400EAC280E4FEC28100D281000EEEB404F56C
:1093B400E4FEEF30E704D2808002C280C28100D292
:1093C40081001237F7B404EAC280E4FEC28100D2FD
:0A93D40081000EEEB404F502A92F8B
:10A7AC00EF1FAC0670011E4C6010E4F5D875F9FC77
:0BA7BC0075E966D2DE20DFE880FB229A
:10A92F00E4FF000000000000000000000FEFB46E15
:01A93F00F126
:01A9400022F4
:102A7E00EC4D6011E8497017ED33EC3304600DE452
:102A8E00FCFFFEFD22E933E8330470F8022CCE126F
:102A9E002C9958046009E4CC248150062850090270
:102AAE002CD8284003022CD5C0E0EB4A7044B980E4
:102ABE0006D0E0FB022CC4EF4E701CBD8008EBFF6D
:102ACE00EAFEE9FD80EBE98DF0A4FEE5F0022B674E
:102ADE00E9CDF9EAFEEBFFEF89F0A4FCE5F0CE8933
:102AEE00F0A42EFFE435F0CD89F0A42DFEE435F0F0
:102AFE008067EF4E7005BD80D780C3EF8BF0A4AC1E
:102B0E00F0EE8BF0A42CFCE435F0F8EF8AF0A42C58
:102B1E00E5F038FCE433CB8DF0A42CFCE5F03BF86B
:102B2E00EE8AF0A42CFCE5F038F8E433CF89F0A45B
:102B3E002CFCE5F038CF3400CE89F0A42FFFE5F061
:102B4E003EFEE433C98DF0A42EFEE5F039CD8AF0B9
:102B5E00A42FFFE5F03EFEE43DFD33D0E0FB500731
:102B6E000BBB000F022CD8EC2CFCEF33FFEE33FE28
:062B7E00ED33FD022CB056
:102B8400022CD8EC5D046005E859047003022CCED5
:102B9400122C99580460F6EC4860F2EC7004FDFEC7
:102BA400FF22C860DB2481C85009C3986002500624
:102BB400022CD59850CAF582E9294B4A7005AB829C
:102BC400022CC475F0007C1A7880C3EF9BEE9AED5A
:102BD40099400DC3EF9BFFEE9AFEED99FDE842F09C
:102BE400DC23ACF0D0E0FFD0E0FED0E0FDAB8220EF
:102BF400E7101BEB60BAEC2CFCEF33FFEE33FEED79
:102C040033FD022CB0E803F830E705C0F075F0009E
:102C1400EF2FFFEE33FEED33FD40B830E7C280AA5C
:102C240075F020800E75F010800575F0087D007E2B
:102C3400007F003392D530D50312302AEC33401094
:102C4400EF33FFEE33FEED33FDEC33FCD5F0ED2234
:0E2C5400E5F0247EA2D513CC92E7CDCEFF2270
:102C6200EDD2E7CD33EC3392D524814006E4FFFE6A
:102C7200FDFC22FCE4CFCECDCC24E0501174FF80C9
:102C8200EDC3CC13CCCD13CDCE13CECF13CF047066
:072C9200F030D5DE02302A0C
:1062CE003A70FA83BCAAE9E43E81E0F8BF9DE9E6A4
:1062DE003F80000039283C1ABB9969663DA335E31F
:1062EE00BF255DE73FC90FDB418DDBCCC44936EEE0
:1062FE0045C9913FC5B0F83D3F800000C317F53446
:10630E00452FFA73C60AFDDD1263D704A2E1921A75
:10631E001420E0159062CE7404122DDB80301263CF
:10632E00D730E102B21A20E0EBA883A982900225B1
:10633E00123075898288839062E27404122DDB8597
:10634E0082F090022512305985F082122A7EED4C91
:10635E006007301A04EC6480FC221263D7C0E0A8F8
:10636E0083A98290022512307589828883906306F4
:10637E007403122DDB8582F090022512305985F0C0
:10638E0082122A7E900225E0CCF0A3E0CDF0A3E0AD
:10639E00CEF0A3E0CFF09062F67403122DDBD08224
:1063AE008582F090022512305985F082E58230E028
:1063BE0007122B87B21A8096EFCBFFEECAFEEDC9FD
:1063CE00FDECC8FC122B878085ED33EC547FCC336B
:1063DE00921A24605007D0E0D0E0022CCE7B837A54
:1063EE00F97922783E122A7EEDF933ECF8332481C6
:1063FE005011EFFBEEFA122C62122C24ECB2E7FCD9
:10640E00122CEAED33EC33602F2403F8C313FCEDAA
:10641E0092E7FDE82481E4501FECF8EDF9EEFAEF77
:10642E00FB122C62EF04C2E0FCF582122C2EECB2B1
:10643E00E7FC122CEAE58203FAED33EC3360071425
:08644E0013FCED92E7FDEA22C8
:102C9900E9D2E7C933E833F892D5EDD2E7CD33EC81
:072CA90033FC5002B2D522FA
:102CB000EC30E7100FBF000C0EBE00080DBD000485
:102CC0000BEB6014A2D5EB13FCED92E7FD2274FF31
:102CD000FCFDFEFF22E480F8A2D574FF13FC7D808A
:032CE000E480EF9E
:102CE300022CCEE86480F8E933E83360110460F025
:102CF300ED33EC337009E8FCE9FDEAFEEBFF220457
:102D030060DED3EB9FEA9EE99DE8C2E78CF0C2F751
:102D130095F0400CE8CCF8E9CDF9EACEFAEBCFFB1D
:102D2300122C9985D0F05804700320D5B3E80470B1
:102D3300075002B2D5022CD892D5EC0460F7E4CC4C
:102D4300C0E0C398F8603B94186008400DD0E0FBE6
:102D5300022CB0E4FBFAC9FC8028E830E406E4C99D
:102D6300FBE4CAFCE830E305E4C9CACBFCE854073A
:102D73006010F8C3E913F9EA13FAEB13FBEC13FC45
:102D8300D8F130F52FC3E49CFCEF9BFFEE9AFEEDE8
:102D930099FDD0E0FBEF4E4D4C701222DB03022C69
:102DA300D5EC2CFCEF33FFEE33FEED33FDED30E7D6
:102DB300EB022CB0EF2BFFEE3AFEED39FDD0E0FB3A
:102DC30050130BBB0003022CD8ED13FDEE13FEEFE3
:082DD30013FFEC13FC022CB00D
:102DDB00C0E0EFFBEEFAEDF9ECF8122A7ED0E0F54D
:102DEB00F0EFFBEEFAEDF9ECF8123049A3A3A3A335
:102DFB00E8C0E0E9C0E0EAC0E0EBC0E0C0F0122AB6
:102E0B007E123065A3A3A3A3122CEAD0F0D0E0FB73
:0D2E1B00D0E0FAD0E0F9D0E0F8D5F0D422F4
:0300000002AA2D24
:0CAA2D00787FE4F6D8FD75812302A8773D
:102E2800BB010689828A83E0225002E722BBFE02A8
:092E3800E32289828A83E49322DB
:102E4100BB010CE58229F582E5833AF583E0225046
:102E510006E92582F8E622BBFE06E92582F8E22290
:0D2E6100E58229F582E5833AF583E49322AA
:102E6E00F8BB010DE58229F582E5833AF583E8F09A
:102E7E00225006E92582C8F622BBFE05E92582C846
:022E8E00F2222E
:102E9000EF8DF0A4A8F0CF8CF0A428CE8DF0A42E56
:022EA000FE2210
:102EA200BC000BBE0029EF8DF084FFADF022E4CC14
:102EB200F875F008EF2FFFEE33FEEC33FCEE9DECDD
:102EC200984005FCEE9DFE0FD5F0E9E4CEFD22ED23
:102ED200F8F5F0EE8420D21CFEADF075F008EF2F6D
:102EE200FFED33FD4007985006D5F0F222C398FD5E
:052EF2000FD5F0EA22FB
:102EF700C5F0F8A3E028F0C5F0F8E5821582700266
:062F07001583E038F02202
:102F0D00E88FF0A4CC8BF0A42CFCE98EF0A42CFC63
:102F1D008AF0EDA42CFCEA8EF0A4CDA8F08BF0A4E1
:102F2D002DCC3825F0FDE98FF0A42CCD35F0FCEB40
:102F3D008EF0A4FEA9F0EB8FF0A4CFC5F02ECD3905
:0F2F4D00FEE43CFCEAA42DCE35F0FDE43CFC2272
:102F5C0075F008758200EF2FFFEE33FECD33CDCC2C
:102F6C0033CCC58233C5829BED9AEC99E5829840AF
:102F7C000CF582EE9BFEED9AFDEC99FC0FD5F0D68C
:102F8C00E4CEFBE4CDFAE4CCF9A88222B800C1B9B6
:102F9C000059BA002DEC8BF084CFCECDFCE5F0CBF4
:102FAC00F97818EF2FFFEE33FEED33FDEC33FCEB2D
:102FBC0033FB10D703994004EB99FB0FD8E5E4F9E8
:102FCC00FA227818EF2FFFEE33FEED33FDEC33FCD5
:102FDC00C933C910D7059BE99A4007EC9BFCE99AC9
:102FEC00F90FD8E0E4C9FAE4CCFB2275F010EF2F0E
:102FFC00FFEE33FEED33FDCC33CCC833C810D7070E
:10300C009BEC9AE899400AED9BFDEC9AFCE899F848
:0E301C000FD5F0DAE4CDFBE4CCFAE4C8F922DB
:0E302A00C3E49FFFE49EFEE49DFDE49CFC22B7
:10303800EB9FF5F0EA9E42F0E99D42F0E89C45F0EE
:013048002265
:10304900E493FC740193FD740293FE740393FF22CD
:0C305900E0F8A3E0F9A3E0FAA3E0FB22FA
:10306500E493F8740193F9740293FA740393FB22C1
:0C307500ECF0A3EDF0A3EEF0A3EFF022CE
:10308100A8828583F0D083D08212309812309812B2
:103091003098123098E473E493A3C583C5F0C583D7
:1030A100C8C582C8F0A3C583C5F0C583C8C582C899
:0130B10022FC
:00000001FF
